:020000040800F2
:1000000000800020437E0008F77F0008B97E0008CA
:10001000F77F0008F77F0008F77F00080000000066
:10002000000000000000000000000000F77F000852
:10003000F77F000800000000F77F0008691500083E
:10004000F77F0008F77F0008F77F0008F77F0008B8
:10005000F77F0008F77F0008F77F0008F77F0008A8
:10006000F77F0008F77F0008F77F0008F77F000898
:10007000F77F0008F77F0008F77F0008F77F000888
:10008000F77F000800000000F77F0008F77F0008F6
:10009000F77F0008F77F0008F77F0008F77F000868
:1000A000F77F0008F77F0008F77F0008F77F000858
:1000B000F77F0008F77F0008F77F0008F77F000848
:1000C000F77F0008F77F0008F77F0008F77F000838
:1000D000F77F0008F77F000801160008F77F000887
:1000E000F77F0008F77F0008F77F0008F77F000818
:1000F000F77F0008F77F0008F77F00080000000086
:1001000000000000F77F000800000000F77F0008F3
:10011000F77F000800000000F77F0008F77F000865
:10012000F77F0008F77F0008F77F0008F77F0008D7
:10013000F77F00080000000000000000F77F0008C3
:10014000F77F0008F77F00080000000000000000B3
:10015000000000000000000000000000000000009F
:10016000000000000000000000000000F77F000811
:10017000F77F000800000000000000000000000001
:1001800000000000F77F00080000000000000000F1
:10019000000000000000000000000000000000005F
:1001A0000000000000000000F77F0008F77F000853
:1001B000F77F0008F77F0008F77F000800000000C5
:1001C00000000000F77F00080000000000000000B1
:0801D000F77F0008F77F00082B
:1001D8002DE9F0411C4B1E683768384607F052FA83
:1001E800044656F8048C404607F04CFA214607F0BE
:1001F80021F907F05FFA04460D460FA3D3E900235F
:1002080007F0EEF980B90EA3D3E90023204629466A
:1002180007F002FA40B908FB07F746F8047C0A4AD7
:100228001368043B136004E0084A136843F48063CE
:100238001360BDE8F08100BF0000C0FFFFFFDF4191
:100248000000C0FFFFFFDFC194680020D0680020D5
:100258002DE9F047344B1C682568002D44D054F82C
:10026800088C54F8049C484607F00CFA06464046A9
:1002780007F008FA314607F0DDF8824607F01AFA67
:1002880006460F4624A3D3E9002307F0A9F938B995
:1002980023A3D3E900233046394607F0BDF980B3DC
:1002A800284607F0EFF90146504607F029F90546B8
:1002B80007F000FA06460F4617A3D3E9002307F014
:1002C8008FF9C0B916A3D3E900233046394607F0A1
:1002D800A3F980B9A4F10802134B1A60284607F065
:1002E800B7F944F8080C04E0104A136843F40063B3
:1002F8001360BDE8F0870D4A136843F48063136008
:10030800F7E7A4F10802084B1A6009FB08F898FB04
:10031800F5F544F8085CECE70000C0FFFFFFDF419B
:100328000000C0FFFFFFDFC194680020D0680020F4
:1003380008B5284B9A6D42F080529A651A6842F4C3
:1003480080321A604FF4A02322490A6812F4003F51
:1003580002D1013BF9D13CE01F4B40F202721A6016
:10036800A3F580539A689A609A689A609A689A6026
:100378004FF48062DA60D3F8882022F04062C3F834
:100388008820D3F8882042F00062C3F88820DA6811
:1003980042F08872DA60DA6842F00302DA601A68BA
:1003A80042F080721A601A46136813F0007FFBD07F
:1003B800084A936843F003039360936803F00C03BF
:1003C8000C2BFAD101F074F9024A936C43F4807350
:0C03D800936408BD0010024000200240A9
:1003E400332303494AF6AA220A60013BFCD1704731
:0403F4000030004095
:1003F8000B4B1B686BB90A4B32221A60094B4AF641
:10040800AA221A60084B1B6823B1013B064A1360F5
:1004180003B170474FF0904320229A61F9E700BF7B
:0C0428000869002000300040106900202E
:10043400054B186038B110B51C46FFF7DBFF236885
:0C044400002BFAD110BD70471469002095
:1004500008B504F0CFF8104AD2F80038D2F80428D2
:100460001340B3F1FF3F13D00B4BD3F81038DB43ED
:100470000A4A13600A2B04D0102B02D013460A221A
:100480001A60054BD3F81438DB43054A136003B1F7
:1004900008BD04F0AFF8FBE700B00008340200200C
:0404A0000C690020C3
:1004A40008B5444B186910F48030FBD1414B5B69AB
:1004B400002B70DA3F4B404A9A6002F188329A600E
:1004C400A3F5F8334AF6AA221A603A4A136913F4D8
:1004D400803FFBD1374B394A5A615A6942F4803222
:1004E4005A61186910F48030FBD1324B1A6942F01A
:1004F40001021A611B6913F0020F4CD12D4B5A698A
:1005040022F002025A615A6942F001025A612C4BEC
:100514000022C3F80028A2F28442C3F80428254B21
:10052400186910F48030FBD1224B1A6942F00102A1
:100534001A611B6913F0020F2DD1214B214AC3F814
:1005440008286FF00B02C3F80C281A4B186910F432
:100554008030FBD1174B1A6942F001021A611B6902
:1005640013F0020F17D1184B1B68154AC2F8103844
:10057400164B1B68DB43C2F814380E4B186910F491
:100584008030FBD10B4B1A6942F001021A611B69DE
:1005940013F0020F00D008BD064B5A6922F0010285
:1005A4005A615A6942F000425A610A20FFF740FF3B
:1005B4000120F0E70020024023016745BA00000350
:1005C40000B00008BFA8FFFF340200200C6900201F
:1005D400164A936D43F4003393654FF090431A68C1
:1005E40022F050021A601A6842F0A0021A601A6AD5
:1005F40022F47F421A621A6A42F4EE421A620C4BE7
:100604000C4A13600C4A13600C4B0D4A13600D4ADC
:1006140013600D4B4FF4D072DA6000225A609A6076
:100624002D221A60094B40225A6070470010024084
:100634004C61002000690020FC6800200842002072
:10064400F8680020F46800200044004000E100E065
:1006540038B5114B1A68511C196010701A680F4B89
:100664001B689A4213D00E4A136843F08003136048
:100674000C4D094CFFF7BEFE2B682268934288BFDD
:1006840002F57A62D31AB3F5756FF3D838BD024B0D
:10069400054A1A60E7E700BFF86800203C02002022
:0C06A40000440040F468002008420020E0
:1006B00070B5744B1B68002B00F0C68003F5005327
:1006C00002339C032368B3F1FF3F2ED06368DB4302
:1006D0006D4A13600A2B04D0102B02D013460A2255
:1006E0001A60694B1A68694B1A60A368DB43684A51
:1006F0001360E368DB43C3F30161664A1160C3F32F
:100700000541654A11609BB2644A13602269D24375
:10071000634B1A606369DB43190C09D04FF6FF7015
:10072000814205D05F48016006E003F063FF8BE083
:100730005C494FF0FF3008609BB233B14FF6FF7158
:100740008B4202D058490B6003E0574B4FF0FF310A
:1007500019606AB9A369DB43544A1360E269D24362
:100760000DD04FF6FF718A4209D051490A600AE064
:1007700004F052F904F0CAF904F04CFAEAE74C4AE2
:100780004FF0FF31116033B904F1300C494C04F5DE
:10079000FC65A64612E004F0EBFA04F04BFBF3E72D
:1007A0000B68DB43CEF810304B68DB43CEF81430D7
:1007B0000CF1180C0EF1180EAE4510D0ACF1100172
:1007C000724651F8043BDB431370180A5070180C42
:1007D00090701B0ED37004326145F2D1E0E7294BD3
:1007E0001B68013B9D03344A02EB833C334E04F506
:1007F0007C640AE00B68DB4333614B68DB43736165
:100800000CF1180C1836A64210D0ACF1100132468B
:1008100051F8043BDB431370180A5070180C9070A9
:100820001B0ED37004326145F2D1E3E7244B03F58C
:100830004050C3F1006101F55041EA185258D243CB
:1008400043F8042F9842F8D1FFF7CCFD01F036FFB2
:100850000F4B1B683BB11B4B1B6913F4005F02D0AD
:100860000B4B00221A600D20FFF7F4FE02F01EFC75
:10087000074B1B6803B970BD013B134A136006F0B8
:1008800011F9F8E70C690020340200205C680020B0
:10089000F06800207C6800208468002080680020C8
:1008A000C8680020AC680020A8680020C468002048
:1008B000A46800204832002010C80008403A0020F8
:0C08C0004402002000080048A06800204E
:1008CC0008B5434B9A6D42F080529A65DA6C42F04F
:1008DC000102DA64DA6C42F00202DA64DA6C42F099
:1008EC000402DA64DA6C42F00802DA644FF09044E5
:1008FC000025256037480560374A1560374B1D6069
:10090C003749E1604FF0AA31C160D1602026DE602A
:10091C00FFF70CFDE36823F44063E360236823F4E2
:10092C0040632360236843F480632360A6612D4BEE
:10093C0032221A602C4B1D602C4B1D602C4B1D6001
:10094C002C4B1D602C4B2D4A1A600A232C4A136029
:10095C002C4A13602C4B1B682C4AA2FB03239B09CB
:10096C00013BB3F1807F09D24FF0E0225361284B59
:10097C00F02183F823109561072313616420FFF79E
:10098C0053FD244C45F2555323604FF6FF73A3607F
:10099C000220FFF749FD022565602846FFF744FD5C
:1009AC004CF6CC432360FFF74DFDFFF70DFE2846B8
:1009BC00FFF73AFDFFF776FE174C02F019FE05F033
:1009CC0083FC2368002BF8D006F0D6F8F5E700BFBF
:1009DC00001002400004004800080048000C0048C9
:1009EC00AAAA02A40869002010690020146900203A
:1009FC00046900200C69002098680020A1B0B9128D
:100A0C00340200205C68002044020020D34D6210A8
:0C0A1C0000ED00E00030004050680020B9
:100A2800914B1B68002B00F054842DE9F0478CB0E3
:100A38008E4A136913F4803FFBD18C4B5B69002B02
:100A4800C0F2AA808A4B4AF6AA221A602E20FFF723
:100A5800FDFD854B1C68013CE400844A136913F4CE
:100A6800803FFBD104F11803DB0043F0407343F0EF
:100A780002037E4A5361536943F48033536113463A
:100A8800186910F48030FBD1784B1A6942F00102E2
:100A98001A611B6913F0020F40F0FC83734B5A690B
:100AA80022F002025A6104F580321832D2025969E2
:100AB80041F001015961002313606E4B1B68DB4351
:100AC80053606A4B186910F48030FBD1674B196981
:100AD80041F0010119611B6913F0020F40F0DA833C
:100AE800654B1B68DB439360644B1968644B1B6858
:100AF8001B0443EA0163634909680B43DB43D36082
:100B08005A4B186910F48030FBD1584B196941F0E1
:100B1800010119611B6913F0020F40F0BB835A4BA6
:100B28001B68DB431361594B1968594B1B8843EA0F
:100B38000143DB4353614D4B186910F48030FBD1FE
:100B48004A4B196941F0010119611B6913F0020F41
:100B580040F0A0834F4B1B68DB4393614E4B1968F1
:100B68004E4B0B40DB43D361404B186910F4803087
:100B7800FBD13E4B196941F0010119611B6913F062
:100B8800020F40F087832032454F07F5FC6EBC46C4
:100B980004AE0AAD354B0AE0344B424A9A6002F182
:100BA80088329A604EE70CF1300CF4457CD0E84668
:100BB800604690F801908178090441EA092190F88B
:100BC800009041EA090190F8039041EA096148F868
:100BD800041B0430B045ECD16046DCF810100491D9
:100BE800DCF8141005910DF11809E04698F819A0E1
:100BF80098F81A10090441EA0A2198F818A041EA5D
:100C08000A0198F81BA041EA0A6149F8041B08F197
:100C18000408A945EAD1816A0A91C16A0B9102F1D7
:100C2800080802F1380AE9464246D9F80010C943D3
:100C380048F8081CD9F80410C94348F8041C186976
:100C480010F48030FBD1196941F00101196119696B
:100C580011F0020F40F01E8308F1080809F1080995
:100C6800D045E1D19FE700BF0C6900200020024079
:100C78000030004034020020F06800207C6800202A
:100C88008468002080680020C8680020AC680020C4
:100C9800A8680020C4680020A468002000F0FF0FA6
:100CA8004832002023016745564A536923F001035F
:100CB8005361554B4AF6AA221A602E20FFF7C6FC4C
:100CC800504A136913F4803FFBD14E4B5B69002BEC
:100CD80034DB4C4A136913F4803FFBD104F1190348
:100CE800DB0043F0407343F00203464A5361536903
:100CF80043F4803353611346186910F48030FBD1F4
:100D0800404B1A6942F001021A611B6913F0020F85
:100D180040F0C0823B4B5A6922F002025A6104F546
:100D2800803808F119084FEAC828C4465A6942F0C1
:100D380001025A61354907F57C6709E0314B344AAD
:100D48009A6002F188329A60C3E73031B94261D0C3
:100D5800EE46084690F801908278120442EA092289
:100D680090F8009042EA090290F8039042EA09627A
:100D78004EF8042B0430B645ECD108460A690492B3
:100D88004A6905920DF118098E469EF819A09EF839
:100D98001A20120442EA0A229EF818A042EA0A021D
:100DA8009EF81BA042EA0A6249F8042B0EF1040ED1
:100DB800A945EAD1826A0A92C26A0B920CF1080E1E
:100DC8000CF1380AE946F446D9F80020D2434EF827
:100DD800082CD9F80420D2434EF8042C186910F4D2
:100DE8008030FBD11A6942F001021A611A6912F0C7
:100DF800020F40F04F820EF1080E09F10809D6459E
:100E0800E1D1A2E70020024000300040283A00204B
:100E180023016745A84A536923F001035361A74B8F
:100E28004AF6AA221A602E20FFF710FCA24B1A6974
:100E380012F4803FFBD1A04B5B69002BC0F22D82DE
:100E48009D4B1A6912F4803FFBD104F11A03DB00B1
:100E580043F0407343F00203974A5361536943F4E4
:100E6800803353611346186910F48030FBD1924BDC
:100E78001A6942F001021A611B6913F0020F40F06F
:100E880009828D4A536923F00203536108F5006310
:100E9800516941F00101516108F580558849A1EB7C
:100EA80008010F1DC858C0431860F858C04358605F
:100EB8000833106910F48030FBD1166946F001063A
:100EC8001661166916F0020F40F0E4819D42E9D1DF
:100ED800794A536923F001035361784B4AF6AA22F1
:100EE8001A602E20FFF7B2FB734B1A6912F4803F89
:100EF800FBD1714B5B69002BC0F2D6816E4B1A692E
:100F080012F4803FFBD104F11B03DB0043F0407374
:100F180043F00203684A5361536943F480335361D1
:100F28001346186910F48030FBD1634B1A6942F0FC
:100F380001021A611B6913F0020F40F0AB815E4B8E
:100F48005A6922F002025A615A6942F001025A6152
:100F58005C4A08F5C056D2F80018C9432960D2F88F
:100F68000418C94369600835186910F48030FBD14A
:100F7800196941F001011961196911F0020F40F076
:100F880089810832AE42E6D14B4A536923F0010306
:100F980053614A4B4AF6AA221A602E20FFF756FBE5
:100FA800454B1A6912F4803FFBD1434B5B69002B18
:100FB800C0F28181404B1A6912F4803FFBD104F1E1
:100FC8001C03DB0043F0407343F002033A4A5361C9
:100FD800536943F4803353611346186910F4803021
:100FE800FBD1354B1A6942F001021A611B6913F0F3
:100FF800020F40F04F81304B5A6922F002025A61C9
:101008005A6942F001025A612F4A08F500551168E1
:10101800C94331605168C94371600836186910F4D2
:101028008030FBD1196941F001011961196911F08A
:10103800020F40F02F810832B542E8D11E4A5369A9
:1010480023F0010353611D4B4AF6AA221A602E2091
:10105800FFF7FCFA184B1A6912F4803FFBD1164BC4
:101068005B69002BC0F22E81134B1A6912F4803F82
:10107800FBD104F11D03DB0043F0407343F002038E
:101088000D4A5361536943F4803353611346186919
:1010980010F48030FBD1084B1A6942F001021A6142
:1010A8001B6913F0020F40F0F580034B5A6922F0D8
:1010B80002025A615A6909E00020024000300040EB
:1010C80048FAFF1F480200204812002042F001029F
:1010D8005A61814A08F520561168C9432960516848
:1010E800C94369600835186910F48030FBD1196963
:1010F80041F001011961196911F0020F40F0CA802D
:101108000832AE42E8D1754A536923F001035361AE
:101118002E20FFF79BFA714B1A6912F4803FFBD11E
:101128006E4B5B69002B05DA6C4B6D4A9A6002F1D5
:1011380088329A60694B1A6912F4803FFBD104F136
:101148001E03DB0043F0407343F00203634A53611C
:10115800536943F4803353611346186910F480309F
:10116800FBD15E4B1A6942F001021A611B6913F048
:10117800020F40F08F80594B5A6922F002025A61DF
:101188005A6942F001025A61564A08F540551168F9
:10119800C94331605168C94371600836186910F451
:1011A8008030FBD1196941F001011961196911F009
:1011B800020F6FD10832AE42E9D1484A536923F091
:1011C80001035361484B4AF6AA221A602E20FFF702
:1011D8003DFA424B1A6912F4803FFBD13F4B5B69E1
:1011E800002B05DA3D4B3E4A9A6002F188329A603C
:1011F8003A4B1A6912F4803FFBD104F11F03DB005C
:1012080043F0407343F00203344A5361536943F493
:10121800803353611346186910F48030FBD12F4B8B
:101228001A6942F001021A611B6913F0020F31D1E9
:101238002A4B5A6922F002025A615A6942F00102A5
:101248005A612A4A08F560581168C94329605168EB
:10125800C94369600835186910F48030FBD11969F1
:1012680041F001011961196911F0020F12D1083218
:10127800A845E9D1194C636923F0010363612E2065
:10128800FFF7E4F9636943F0004363610A20FFF75D
:10129800CDF801200CB0BDE8F087104B104A9A60D9
:1012A80002F188329A60CBE50C4B0D4A9A6002F144
:1012B80088329A6022E6094B094A9A6002F188321C
:1012C8009A6077E6054B064A9A6002F188329A607E
:1012D800CAE60120704700BF481A002000200240DB
:1012E800230167454822002000300040482A00209A
:1012F80010B5041E7ADB092C72D9632C64D9B4F5B5
:101308007A7F56D342F20F739C4246D9404B9C4297
:1013180037D9404B9C4228D93F4B9C421AD33F4B6C
:101328009C420CD93E4B9C4265D83E48A0FB0430F9
:10133800400E3D4B03FB10443030FFF787F93B4824
:10134800A0FB0430800D344B03FB10443030C0B296
:10135800FFF77CF93648A0FB0430800C354B03FBC3
:1013680010443030C0B2FFF771F96009324BA3FB6B
:101378000030C009314B03FB10443030C0B2FFF7D6
:1013880065F92F48A0FB0430400B42F2107303FBB1
:1013980010443030C0B2FFF759F92A48A0FB043096
:1013A80080094FF47A7303FB10443030C0B2FFF762
:1013B8004DF92548A0FB04304009642303FB104481
:1013C8003030C0B2FFF742F92048A0FB0430C00813
:1013D80000EB8003A4EB43043030C0B2FFF736F9CA
:1013E80004F13000C0B2FFF731F910BD2D20FFF72E
:1013F8002DF964427FE7600A154BA3FB0030C00952
:10140800144B03FB10443030FFF720F98DE700BF81
:101418009F8601003F420F0080969800FFE0F50587
:10142800FFC99A3B893BE65500E1F5056BCA5F6B3E
:1014380083DE1B4340420F00C55A7C0AA086010088
:101448005917B7D1D34D62101F85EB51CDCCCCCCF9
:08145800834B040000CA9A3B1B
:1014600010B594B00DF1300C244C0FCCACE80F004B
:1014700094E80F00ACE80700ACF800300DF1140C54
:101480001F4C0FCCACE80F0094E80700ACE8030059
:101490008CF800201B4B01AC0FCB07C424F8023B97
:1014A0001B0C23700D20FFF7D5F80CA806F01BFFCE
:1014B0003120FFF7CFF82E20FFF7CCF81220FFF7EE
:1014C0001BFF01A806F00FFF0F4B18680F4BA3FB83
:1014D0000030800CFFF710FF4D20FFF7BBF84820CD
:1014E000FFF7B8F87A20FFF7B5F805A806F0FBFE7D
:1014F0000D20FFF7AFF814B010BD00BF6C800008DE
:101500008C800008A88000084402002083DE1B4372
:1015100008B5FEF771FF0F4B1B680F4A1268934224
:1015200015D05A1C0B490A60187840F400400B4B48
:101530001B689A4208D04FF090434FF400129A6112
:10154000074B04221A6008BD064A0A60F3E7002030
:10155000F9E700BFFC68002000690020400200207D
:08156000106900204C6100201D
:101568001C4B1B6813B1013B1A4A13601A4B1B68CA
:1015780013B1013B184A1360184B1B6813B1013BA8
:10158800164A1360164B1B6813B1013B144A1360CB
:10159800144B1B6813B1013B124A1360124B1B68B2
:1015A80013B1013B104A1360104B1B6813B1013B88
:1015B8000E4A13600E4B1B6813B1013B0C4A1360B3
:1015C8000C4A136883EA433383EA534383EA431399
:1015D800136070470869002014690020046900201E
:1015E800B868002060680020906800208C6800209F
:0815F8008868002098680020BB
:1016000008B5204BDB6913F0200F10D01D4B5B6A2F
:10161000DAB2022A21D0042A27D01B4A11680B70A3
:10162000136801331360194A1268934219D0154B9D
:10163000DB6913F0800F0FD0154B1B68154A126839
:10164000934215D05A1C12490A6019780D4B9962C1
:10165000114B1B689A4211D008BD104A022111603B
:10166000DBE7094B0E4A1A60E1E701F045FADEE7D5
:10167000044A136823F080031360EDE7044B094A22
:101680001A60E9E7004400400069002040020020A1
:10169000F4680020F86800203C0200205468002014
:0816A0004C610020084200200B
:1016A800024B4FF000629A60704700BF00ED00E007
:1016B8001D4B9B6803F00C03082B12D00C2B14D085
:1016C800042B0AD0184B9B68184AC3F30313184914
:1016D800C95C1368CB4013607047144B154A1A60F5
:1016E800F0E7124B144A1A60ECE70F4BDA68DB6834
:1016F800C3F30313013302F00302022A0CBF0D499E
:101708000D49B1FBF3F1084AD368D268C3F3062345
:1017180001FB03F3C2F3416201325200B3FBF2F35F
:10172800024A1360CEE700BF0010024044020020C6
:0C173800F07600080024F40000366E017A
:10174400024A136843F0200313607047D0680020F6
:10175400064A1368043B1360054A934204D2054ABF
:10176400136843F004031360704700BF94680020BB
:081774005C660020D068002033
:10177C0007490B681A1D0A6006498A4202D21A6888
:10178C005A607047044A136843F0040313607047AF
:0C179C009468002040670020D068002006
:1017A800044A136853F8041C186843F8040C1368B7
:0817B8001960704794680020DD
:1017C000034A1368191D116053F8042C5A607047BE
:0417D00094680020F9
:1017D400074B1A6852F8081C52F8040C42F8080C1B
:1017E4001A68106842F8040C1B681960704700BF3F
:0417F40094680020D5
:1017F800074B1A68116852F8040C10601A6852F8FE
:10180800080C42F8040C1B6843F8081C704700BF1A
:0418180094680020B0
:10181C000D4B1B681A680D49591A6FF00300801A9A
:10182C0010EBA10105D452B1A3EB820212681A602D
:10183C007047074A136843F0040313607047043B76
:10184C00014A1360704700BF946800205066002066
:04185C00D068002030
:10186000164B1B681968164A9A1A6FF00300401A43
:1018700010EBA2021AD4043B104A136001291BD9B1
:1018800030B4C1F1010253F82250C1F102029200BA
:101890000A4C23689858134443F8040C0432013965
:1018A000F7D1064B1B681D6030BC7047054A1368B2
:1018B00043F0040313607047704700BF9468002032
:0818C00050660020D0680020F2
:1018C80070B4164B1B681D68154A9A1A6FF003010D
:1018D800491B11EBA2021BD453F8046D0F4A136085
:1018E800012D13D905F1FF3C6FF0030200210B4CC9
:1018F80023689858134458600131043A6145F7D178
:10190800C5F10105054B1B6843F8256070BC70479D
:10191800044A136843F004031360F7E7946800204F
:0819280050660020D068002089
:10193000054B1A6852F8041C1068014442F8041C54
:0C1940001A68043A1A607047946800208E
:10194C00024B1A68136801331360704794680020C7
:10195C00054B1A6852F8041C1068091A42F8041C4A
:0C196C001A68043A1A6070479468002062
:10197800024B1A681368013B136070479468002093
:10198800034B1A681368002BBCBF5B421360704797
:04199800946800202F
:10199C000F4B1B681A6882EAE270A0EBE2701F28FA
:1019AC0010DC10B4191F0A4C2160002AA7BF53F891
:1019BC00041C01FA02F253F8042CC24043F8042C24
:1019CC0010BC7047034A136843F48063136070477C
:0819DC0094680020D06800208F
:1019E400054B1A6852F8041C1068014042F8041CA4
:0C19F4001A68043A1A60704794680020DA
:101A0000054B1A6852F8041C1068014342F8041C84
:0C1A10001A68043A1A60704794680020BD
:101A1C00054B1A6852F8041C1068414042F8041C2B
:0C1A2C001A68043A1A60704794680020A1
:101A3800024B1A681368DB431360704794680020F0
:101A4800024B1A6813685B42136070479468002061
:101A58000A4B1B681A6852B153F8041C91FBF2F246
:101A680043F8042C054A1368043B13607047044A82
:101A7800136843F400631360704700BF9468002044
:041A8800D068002002
:101A8C000B4B1B681A6862B153F8041C91FBF2F003
:101A9C0002FB101243F8042C054A1368043B136034
:101AAC007047044A136843F400631360704700BF27
:081ABC0094680020D0680020AE
:101AC4000A4B1B681A685AB153F8041C91FBF2F0D4
:101AD40002FB101243F8042C044B1B681860704777
:101AE400034A136843F4006313607047946800204A
:041AF400D068002096
:101AF8000B4B1B681A681F2A0CD8012101FA02F245
:101B080053F8041C114343F8041C054A1368043BAA
:101B180013607047034A136843F480631360704787
:081B280094680020D068002041
:101B30000C4B1B681A681F2A0DD8012101FA02F20A
:101B400053F8041C21EA020143F8041C054A1368F7
:101B5000043B13607047044A136843F480631360C6
:0C1B6000704700BF94680020D06800208F
:101B6C000E4B1B681A681F2A11D810B4012101FAF8
:101B7C0002F2194651F8040D084C216030EA0202B9
:101B8C0014BF0122002243F8042C10BC7047044AF5
:101B9C00136843F480631360704700BF946800209F
:041BAC00D0680020DD
:101BB000034A1368191D1160024A12685A6070477F
:081BC0009468002098680020E1
:101BC800074B1A68116852F8040C814214BF0021AF
:101BD800012142F8041C1A68043A1A60704700BFD1
:041BE80094680020DD
:101BEC00064B1A68116852F8040C091A18BF012127
:101BFC0042F8041C1A68043A1A6070479468002072
:101C0C00034B1A681368B3FA83F35B0913607047CC
:041C1C0094680020A8
:101C2000074B1A6852F8041C10688142D4BF002187
:101C3000012142F8041C1A68043A1A60704700BF78
:041C40009468002084
:101C4400074B1A6852F8041C10688142B4BF002183
:101C5400012142F8041C1A68043A1A60704700BF54
:041C64009468002060
:101C6800074B1A6852F8041C10688142ACBF002167
:101C7800012142F8041C1A68043A1A60704700BF30
:041C8800946800203C
:101C8C00074B1A6852F8041C106881422CBF0021C3
:101C9C00012142F8041C1A68043A1A60704700BF0C
:041CAC009468002018
:101CB000074B1A6852F8041C10688142CCBF0021FF
:101CC000012142F8041C1A68043A1A60704700BFE8
:041CD00094680020F4
:101CD4000B4B1A6813680B4999420BD801F57C61C8
:101CE4008B4207D852F8042C1A60054A1368083B43
:101CF40013607047044A136843F02003136070476D
:0C1D04009468002048320020D0680020C5
:101D1000094B1A6813680949994206D801F57C6194
:101D20008B4202D81B6813607047054A136843F062
:101D300020031360704700BF9468002048320020E1
:041D4000D068002047
:101D4400104B1A6813686BB1B3F57A7F0ADC13F58C
:101D54007A7F07DB002B0BDD013B0B4951F8233065
:101D640013607047094A136843F480631360704733
:101D7400DB4352F8040C044941F82300083A014BB0
:101D84001A60704794680020AC510020D06800208D
:101D9400044B0A221A60044B1B680BB9034B1A60EC
:101DA400704700BF5C680020D46800203402002023
:101DB400044B10221A60044B1B680BB9034B1A60C6
:101DC400704700BF5C680020D46800203402002003
:101DD40006490A6852F804390A602BB104494AF6E4
:101DE400AA220A60013BFCD1704700BF946800201E
:041DF400003000407B
:101DF80005490B6853F80429642000FB02F20348E4
:101E080002600B60704700BF946800206068002083
:101E1800074B4AF6AA221A60064B1A68111D196068
:101E2800054B1B680549A1FB03135B095360704709
:101E38000030004094680020606800201F85EB5146
:101E480010B4314A136853F8044913602F490B68DA
:101E580023F001030B602E4A936D43F4001393653E
:101E68002C4B586840F440705860186820F4702073
:101E78001860186840F420201860586A20F0FF00A5
:101E88005862586A40F044005862D86820F47020BC
:101E9800D860D2F8883023F44053C2F88830630001
:101EA800DBB24B6014F4807F22D00B464FF0A04287
:101EB8000A610969184A0A431A61144B00229A6197
:101EC8004FF4E762DA611A6842F001021A60114BB6
:101ED8001B6913F4807F04D00E4B1B6913F4007F39
:101EE80004D10E4A136843F04003136010BC7047D6
:101EF800064A4FF030431361136943F4C22343F099
:101F080014031361D9E700BF94680020005400400F
:101F180000100240000400480A052400D068002090
:101F2800294A136853F804191360284BC8221A6009
:101F3800274A936913F0050FFBD0254B5A6822F006
:101F48007F7222F441325A605A6842F0007242F4B9
:101F580080325A605A6842F400525A609A6912F004
:101F6800010F09D19A6912F4756FF7D0194A1368ED
:101F780043F0400313607047154BDA6922F4F042CE
:101F880022F007021204120CDA61C9B299629A6946
:101F980012F0010F09D19A6912F4756FF7D00D4A42
:101FA800136843F0400313607047094BDA6922F461
:101FB800F04222F007021204120CDA615A6842F465
:101FC80080425A60704700BF94680020046900206E
:081FD80000540040D068002015
:101FE000374B19680868C24301EB82011960354B11
:101FF000994228D300282CD0334BC8221A60334A88
:10200000936913F0050FFBD0304B5A6822F07F72B2
:1020100022F441325A605A6842EA004242F00072A9
:102020005A605A6842F400525A609A6912F0010FDD
:1020300015D19A6912F4756FF7D0254A136843F0E9
:10204000400313607047224A136843F0040313608F
:1020500070471F4A136843F480631360704700B5EC
:102060001A4AD36923F4F04323F007031B041B0C23
:10207000D3614FF0000C134648F2F87E0CF1010CCE
:1020800051F8042FD2B29A629A6912F0010F0AD164
:102090009A6912F4756FF7D00D4A136843F0400344
:1020A00013605DF804FBDA6902EA0E02DA61844526
:1020B000E4D1064A536843F480435360F1E700BF1C
:1020C000946800205C6600200469002000540040F1
:0420D000D0680020B4
:1020D400294BC8221A60294A936913F0050FFBD0D3
:1020E400264B5A6822F07F7222F440325A605A68B2
:1020F40042F0007242F480625A605A6842F48032BC
:102104005A605A6842F400525A609A6912F0010FF8
:1021140009D19A6912F0100FF7D0194A136843F0E5
:10212400400313607047154AD36923F4F04323F046
:1021340007031B041B0CD36113469A6912F0040FA6
:1021440009D19A6912F4756FF7D00D4A136843F0F8
:10215400400313607047094BDA6922F4F04222F01D
:1021640007021204120CDA6106490A68101D08609D
:102174005B6ADBB25360704704690020005400407E
:08218400D068002094680020DF
:10218C00344B196851F80409196050B3324BC8220A
:10219C001A60324A936913F0050FFBD02F4B5A6823
:1021AC0022F07F7222F440325A605A6842F0007278
:1021BC0042F480625A605A6842EA00425A605A6895
:1021CC0042F400525A609A6912F0010F0FD19A69C9
:1021DC0012F0100FF7D0224A136843F0400313603B
:1021EC0070471F4A136843F480631360704730B51F
:1021FC001A4AD36923F4F04323F007031B041B0C86
:10220C00D3610024A446134648F2F8754FF0010E32
:10221C009A6912F0040F0DD19A6912F4756FF7D008
:10222C002CB90F4A136843F04003136030BD094BBF
:10223C001960F6E7DA692A40DA615A6AD2B241F8D3
:10224C00042F0CF1010C74466045E1D1014B19606F
:10225C00ECE700BF946800200469002000540040A3
:04226C00D068002016
:10227000564B1968564B99422AD30B4653F804091A
:10228000524A136050B3534BC8221A60524A9369A2
:1022900013F0050FFBD0504B5A6822F07F7222F4E6
:1022A00041325A605A6842F480325A605A6842F4A5
:1022B00000525A609A6912F0010F15D19A6912F012
:1022C000100FF7D0454A136843F04003136070477E
:1022D000424A136843F00403136070473F4A13688F
:1022E00043F48063136070473B4BDA6922F4F04299
:1022F00022F007021204120CDA6111F8042C9A621F
:102300000839324B1960344B9A6912F0010F09D128
:102310009A6912F0100FF7D0304A136843F0400367
:10232000136070472C4BDA6922F4F04222F0070266
:102330001204120CDA615A6822F07F7222F44032E1
:102340005A605A6842F0007242F480625A605A68D9
:1023500042EA00425A605A6842F400525A609A694E
:1023600012F0010F09D19A6912F0100FF7D01B4A31
:10237000136843F040031360704730B50024A4464F
:10238000154B48F2F8754FF0010E9A6912F0040FE0
:102390000DD19A6912F4756FF7D02CB90F4A1368F2
:1023A00043F04003136030BD084B1960F6E75A6AEA
:1023B000D2B241F8042FDA692A40DA610CF1010C3B
:1023C00074466045E1D1014B1960ECE79468002048
:1023D0005C6600200469002000540040D0680020A2
:1023E0000A4B1A68136803F140400949884207D82C
:1023F00052F8042C1A60054A1368083B13607047B2
:10240000044A136843F480631360704794680020A3
:08241000000C0610D06800204A
:10241800084B1B681A6802F140400749884202D8F5
:1024280012681A607047054A136843F480631360A2
:10243800704700BF94680020000C0610D068002088
:10244800114B1A68136803F14040104988420ED8AE
:1024580052F8042C1F2A10D8012101FA02F2196837
:1024680011431960084A1368083B13607047084A0B
:10247800136843F4806313607047054A136843F494
:1024880080631360704700BF94680020000C06103A
:04249800D0680020E8
:10249C00114B1A68136803F14040104988420FD859
:1024AC0052F8042C1F2A11D8012101FA02F21968E2
:1024BC0021EA02011960084A1368083B136070474F
:1024CC00074A136843F4806313607047044A136827
:1024DC0043F480631360704794680020000C06106E
:0424EC00D068002094
:1024F000134B1B681A6802F140401249884213D8F6
:1025000053F8041C1F2915D810B4012000FA01F15A
:1025100010681A1F0A4C2260014214BF01220022D7
:1025200043F8042C10BC7047074A136843F48063D7
:1025300013607047044A136843F480631360704764
:0C25400094680020000C0610D0680020F9
:10254C0010B408490A6852F804490748074B1B683D
:10255C0003F18043013B00EB830340F824300A6015
:10256C0010BC70479468002048020020E0680020EE
:10257C00044A1368191D1160034A126852F8042C9E
:0C258C005A607047946800209C68002092
:10259800084B4AF6AA221A60074B1B681A68131FD1
:1025A80052F8042C862A0CBF043B5B68034A13606C
:1025B800704700BF003000409C680020C0680020C1
:1025C800024B1B681A68024B1A6070479C6800200F
:0425D800C0680020B7
:1025DC00064B1B681A6822B9054A12681168054A2D
:1025EC001160043B014A1360704700BF94680020DF
:0825FC009C680020C06800206B
:10260400164B1B681968164A1160164A934218D96A
:10261400154A1268022A07D0043B104A1360134A71
:102624001368013B13607047104A1168104A12681E
:102634009142F1D10E4A002111600B4A032111602D
:10264400EAE7074B00221A60074B1B68022B00D0F5
:102654007047054B03221A60FAE700BF9C6800200C
:10266400C06800205065002038020020B4680020B3
:04267400EC680020EE
:10267800054B00221A605A609A6003F10C00034966
:102688000860DA60704700BF506600209468002038
:0C269800014B03221A607047380200203A
:0C26A400014B01221A6070473802002030
:0C26B000014B00221A6070473802002025
:1026BC0010B50023404A1360404A1360404A13602F
:1026CC00404A1360404A1360404A01211160404A5D
:1026DC001360404A1168404A1160404A117819B1A0
:1026EC0001331832A82BF9D13D4A13603D4AD2F878
:1026FC00FC2F772A4DD03C4940F6FF321446013A64
:10270C0051F8040D772834D0002AF7D1002237492C
:10271C000A6037490A60314A03EB430302EBC303F7
:10272C0002F57C62934228BF00240AD200240021C7
:10273C00304A43F8041B9342FBD340F6FE339C42D1
:10274C000AD82D4B03EB8403002140F6FE3243F8EC
:10275C00041F01349442FAD9284A294B1A600023E9
:10276C001360284A28491160284A1360FFF77EFF3E
:10277C0010BD002ACAD01D4A14601D4A1460174AA5
:10278C0003EB430302EBC30302F57C629342CED30B
:10279C00D3E74FF4406215490A6015490A600F4AA5
:1027AC0003EB430302EBC30302F57C62934238BF95
:1027BC004FF44064BBD3CFE7D8680020D468002026
:1027CC00CC680020E8680020B468002038020020A3
:1027DC0058680020340200205C6800204832002039
:1027EC00B06800204822002044320020E06800201D
:1027FC00DC680020084200204402002050650020C4
:10280C009C680020C068002048020020D06800208E
:10281C00054A1368191D116004490A68101D0860E7
:10282C0052685A60704700BF94680020C06800204E
:10283C00054A1368191D116004490A68101D0860C7
:10284C00526812685A60704794680020C068002073
:10285C00064B1A68111D1960054B196809685268F6
:10286C0011601A68043A1A60704700BFC0680020F3
:04287C00946800203C
:10288000084B1B681A6842B1074A126804320649AD
:102890000A60043B034A13607047034A1268526897
:0C28A000F5E700BF94680020C06800202D
:1028AC00084B1B68196853F8042C9142064A1268AD
:1028BC000CBF0432526804490A60043B014A13609D
:0C28CC00704700BF94680020C068002026
:1028D800084B1B68196853F8042C9142064A126881
:1028E800CCBF0432526804490A60043B014A1360B1
:0C28F800704700BF94680020C0680020FA
:10290400084B1B68196853F8042C9142064A126854
:10291400B4BF0432526804490A60043B014A13609C
:0C292400704700BF94680020C0680020CD
:10293000024B1A6852681A60704700BFC0680020D6
:10294000054A1368191D116004490A68101D0860C2
:1029500052685A60704700BF9C680020C068002021
:102960000C4B1B681B6863B10B4A1368043B136074
:102970000A4A136808331360064A1368043B13605D
:102980007047074B4AF6AA221A60044B1A6852682D
:102990001A60F1E7946800209C680020C06800205D
:0429A00000300040C3
:1029A4000C4B1B681B6863B90B4A1368043B136028
:1029B4000A4A136808331360064A1368043B136019
:1029C4007047074B4AF6AA221A60044B1A685268E9
:1029D4001A60F1E7946800209C680020C068002019
:0429E400003000407F
:1029E800044B4AF6AA221A60034B1A6852681A6006
:0C29F800704700BF00300040C0680020A5
:102A04000B4B1A6802F1100119600A490B6853F85C
:102A1400080CD06053F8040C906053F80C09506013
:102A24000B6005490B68181D08605B6813617047EB
:0C2A34009C68002094680020C06800200E
:102A40001C4B1B6853F8042C53F8080C53F80C1C4F
:102A50000A44002916DB90420CDD174B4AF6AA21E6
:102A60001960144B1B6843F8042C144B1A68526805
:102A70001A607047103B0F4A1360104A13680833FE
:102A80001360704790420CDA0B4B4AF6AA2119608A
:102A9000084B1B6843F8042C084B1A6852681A60EC
:102AA0007047103B034A1360044A136808331360ED
:102AB000704700BF9C68002000300040C0680020C4
:102AC000024A1368043B1360704700BF9C680020F3
:102AD000024A1368103B1360704700BF9C680020D7
:102AE00010B5044C23681878FDF7B4FD2368043B47
:082AF000236010BD9468002072
:102AF80008B50E4B1B6803B108BD2020FDF7A6FDE5
:102B08002D20FDF7A3FD3E20FDF7A0FD4420FDF795
:102B18009DFD4220FDF79AFD4720FDF797FD2020F7
:102B2800FDF794FD014B01221A60E5E73802002009
:102B3800F8B5124A13685D6808331360C5B10024FC
:102B480017460AE026FA04F0C0B2FDF77FFD083404
:102B5800192C28BF0024013D0AD0002CF2D13B6873
:102B680053F8046B3B60F0B2FDF770FD0824F2E700
:102B7800024A1368043B1360F8BD00BFC068002018
:102B880008B5104B1B6883B10F4B1B686BB10F4B1B
:102B98001B68ABB10E4A1368191D11600D4A1278F3
:102BA8005A600A4B00221A600AE0FEF7ADFC0346A1
:102BB8000028FAD006490A68101D0860DBB2536085
:102BC80008BD00BF38020020CC68002058680020EB
:082BD800946800201869002038
:102BE00010B5064C2368186805F0E5FB2020FDF7BA
:102BF00031FD2368043B236010BD00BF94680020B2
:102C000008B50E4B1B68102B07D00D4B1B681868BE
:102C100000F160420B4B9A420CD8094B1B681868B4
:102C200005F0C9FB2020FDF715FD054A1368043B9C
:102C3000136008BDFEF760FBF4E700BF5C6800208E
:082C400094680020FF0B063030
:102C48002DE9F04186B02B4B93E8070006AB03E96A
:102C58000700294B93E803000190ADF808105B20AA
:102C6800FDF7F4FC254B1B68254A93420CD0244AF7
:102C780093420DD319D9151D0424A2F10C06DFF8CF
:102C8800848006F10C0725E001A805F028FB0CE07C
:102C980003A805F024FB1C4B00221A605A609A60B6
:102CA80003F10C0015490860DA605D20FDF7CEFCE1
:102CB8002020FDF7CBFC06B0BDE8F081286805F0C0
:102CC80076FB2020FDF7C2FC01340C4B1B68043551
:102CD800BB42EAD99B1BB4EBA30FE6D82020FDF733
:102CE800B5FCD8F80030102BE8D02868FEF700FBB8
:102CF800E7E700BFD07E0008DC7E0008946800206B
:0C2D08005C6600205C6800205066002023
:102D14002DE9F0472020FDF79BFC3E4B1B68002B60
:102D240071D03D4D00273E464FF02008DFF8ECA05F
:102D3400DFF8E0901AE04046FDF78AFC18E0D5F889
:102D4400053013F0406F24D14046FDF781FC404626
:102D5400FDF77EFC4046FDF77BFC01360137052F6D
:102D64004BD81835D9F80030B3424BD9092EE2D9E3
:102D74003046FEF7BFFA3A20FDF76AFCA5F11004CD
:102D840014F8010F0028DAD0FDF762FCAC42F7D149
:102D9400D5E72820FDF75CFC5620FDF759FC61209F
:102DA400FDF756FC7220FDF753FC4320FDF750FC61
:102DB4006F20FDF74DFC6E20FDF74AFC3D20FDF72A
:102DC40047FCDAF80030102B12D0D5F80100FEF7DA
:102DD40091FA4046FDF73CFC4020FDF739FC681CA5
:102DE40080B205F0E6FA2920FDF732FC0237ABE7A2
:102DF400D5F8010005F0DDFAEBE70D20FDF728FC1E
:102E04000027AEE70FB9BDE8F0870D20FDF720FCE1
:102E1400F9E700BFB0680020573200205C6800204A
:102E240010B5044C2368186805F0A3F82368043B24
:082E3400236010BD946800202A
:102E3C0008B5154B1B681B68B3F5805F0CD2134BA0
:102E4C001B6813F0010F0DD00F4A136853F80409D7
:102E5C000E498860136008BD0D4A136843F4806303
:102E6C001360F8E70B4AD36C43F48033D364074BFD
:102E7C001A6802F001121A601A6842F001021A6014
:102E8C00FDF7AAFAE0E700BF9468002000080050A4
:082E9C00D06800200010024084
:102EA40008B5154B1B681B68B3F5805F0CD2134B38
:102EB4001B6813F4803F0DD00F4A136853F80409BC
:102EC4000E494861136008BD0D4A136843F48063DA
:102ED4001360F8E70B4AD36C43F48033D364074B95
:102EE4001A6802F001121A601A6842F480321A60F9
:102EF400FDF776FAE0E700BF946800200008005070
:082F0400D0680020001002401B
:102F0C002DE9F04F83B0284A6B4692E8030083E822
:102F1C000300184605F0E1F90D20FDF795FB234B56
:102F2C0003F1080703F58D6A4FF000084FF0010913
:102F3C0020264FF0230B24E0FDF786FB013415F817
:102F4C00010B0028F8D1062C05D83046FDF77CFB88
:102F5C000134072CF9D15846FDF776FB484605F0AD
:102F6C00C8F93046FDF770FB3046FDF76DFB09F1F3
:102F7C00010908F10108B8F1050F08D008375745C9
:102F8C000ED03046FDF760FB3D460024D7E70D2000
:102F9C00FDF75AFB3046FDF757FB4FF00008EDE705
:102FAC0003B0BDE8F08F00BF007700083C79000843
:102FBC002DE9F0478CB001AC324D0FCD0FC40FCDC5
:102FCC000FC495E8070003C422802F4B1B6863B124
:102FDC002E4B1B684BB12D4B00221A602C4A1368E8
:102FEC00191D11602B4A12685A60294A136853F84C
:102FFC000459136045F00055274B9D4207D9274AC9
:10300C00136843F4806313600CB0BDE8F0870D20A7
:10301C00FDF71AFB01A805F060F9284604F07DFFC6
:10302C0005F1800803264FF00D0A4FF03A097C2772
:10303C0014E02468200E05F05CF9C4F3074005F099
:10304C0058F9C4F3072005F054F9E0B205F051F932
:10305C003846FDF7F9FA043545450ED02C460136B5
:10306C00042EE6D15046FDF7EFFA284604F055FF42
:10307C004846FDF7E9FA0026DBE70D20FDF7E4FAF8
:10308C00C2E700BFFC7E0008CC680020E868002086
:10309C0094680020E4680020807F0020D068002025
:1030AC0070B5ACB0704B93E803002A90ADF8AC103F
:1030BC00090C8DF8AE106D4B27AE93E8070086E82F
:1030CC0007006B4B93E803002590ADF89810090CA2
:1030DC008DF89A10674A23AB92E8030083E803004B
:1030EC001EAC654D0FCD0FC42B6824F8023B1B0C96
:1030FC002370624A1CAB92E8030083E80300604A29
:10310C0019AB07CA03C31A705E4B93E80300179000
:10311C00ADF86010090C8DF862105B4A14AB07CA4D
:10312C0003C31A70594A11AB07CA03C31A70584B20
:10313C001093584B93E803000E90ADF83C10564A90
:10314C000BAB07CA03C31A70544A08AB07CA03C3B4
:10315C001A70534B93E803000690ADF81C10514ABB
:10316C0003AB07CA03C31A704F4B93E803000190DB
:10317C00ADF80810090C8DF80A10FEF76BF9442015
:10318C00FDF762FA6120FDF75FFA7420FDF75CFA37
:10319C006120FDF759FA2AA805F09FF8434804F07E
:1031AC00BCFE5220FDF750FA6520FDF74DFA742055
:1031BC00FDF74AFA7520FDF747FA7220FDF744FA3D
:1031CC006E20FDF741FA2AA805F087F8384804F07C
:1031DC00A4FE304605F081F8364804F09EFE5520DA
:1031EC00FDF732FA7320FDF72FFA6520FDF72CFA64
:1031FC007220FDF729FA3D20FDF726FA2E4804F03F
:10320C008CFE0D20FDF720FA2C4B1B68F3B123A884
:10321C0005F063F8294B1B68E3B91EA805F05DF8AF
:10322C00274B1B68002B4DD00024234E244D2B68BC
:10323C00013B03EB430306EBC303185D00284DD0A1
:10324C00FDF702FA0134102CF1D147E025A805F066
:10325C0044F8DCE72320FDF7F7F9184B18683030F9
:10326C00C0B2FDF7F1F9D8E7B8800008C0800008BB
:10327C00CC800008D4800008DC800008F0800008B6
:10328C00F8800008048100080C81000818810008EF
:10329C004F464600248100082C8100083881000824
:1032AC00448100084C810008588100085C660020AD
:1032BC005065002048020020483200200C69002094
:1032CC00F06800206E20FDF7BFF96F20FDF7BCF908
:1032DC006E20FDF7B9F96520FDF7B6F90D20FDF765
:1032EC00B3F95320FDF7B0F95020FDF7ADF94920A3
:1032FC00FDF7AAF93D20FDF7A7F9AE4B1868FDF7CD
:10330C00F5FF2C20FDF7A0F9AB4B1B68102B00F040
:10331C009D80AA4B1868FDF7E9FF2C20FDF794F966
:10332C00A74B1868FDF7E2FF0D20FDF78DF91CA8DF
:10333C0004F0D3FFA34B1C68002C40F093800020BA
:10334C00FDF7D4FF19A804F0C8FF9F4B186800289C
:10335C00C0F2B480984B1B68102B00F0B380FDF7C3
:10336C00C5FF17A804F0B9FF984B18680028C0F2E5
:10337C00AC80914B1B68102B00F0AB80FDF7B6FFB7
:10338C0014A804F0AAFF924B1C68002C40F0A480F7
:10339C000020FDF7ABFF11A804F09FFF8D4B1868C0
:1033AC000028C0F2C580844B1B68102B00F0C48031
:1033BC00FDF79CFF0D20FDF747F90EA804F08DFFDB
:1033CC00854B1B6FB3F1FF3F40F0BD804FF0904336
:1033DC005B6913F0020F40F0B28001A804F07DFF8E
:1033EC003120FDF731F90BA804F077FF7A4BD3F8B5
:1033FC008830B3F1FF3F40F0B9804FF090435B69E8
:10340C0013F0100F40F0AE8001A804F066FF3220DC
:10341C00FDF71AF908A804F060FF6F4BD3F8A03041
:10342C00B3F1FF3F40F0B6804FF090435B6913F46B
:10343C00807F40F0AB8001A804F04FFF3320FDF7F4
:10344C0003F90D20FDF700F92CB070BD5B4B18682B
:10345C0004F0ABFF2C20FDF7F7F8594B186804F07B
:10346C00A4FF61E74FF4FA6303FB04F55B4EB6FB74
:10347C00F5F63046FDF73AFF06FB04F0584B594C75
:10348C0003FB00442E20FDF7DFF8B4FBF5F63046C5
:10349C00FDF72CFF05FB164303EB83035B00B3FB2B
:1034AC00F5F005FB103303EB83035B00B3FBF5F383
:1034BC00042B88BF0130FDF719FF43E710A804F077
:1034CC000CFF4EE704F071FF4BE710A804F005FF6A
:1034DC0056E704F06AFF53E74FF4FA6303FB04F575
:1034EC003E4EB6FBF5F63046FDF700FF06FB04F04A
:1034FC003B4B3C4C03FB00442E20FDF7A5F8B4FBE2
:10350C00F5F63046FDF7F2FE05FB164303EB83039D
:10351C005B00B3FBF5F005FB103303EB83035B009F
:10352C00B3FBF5F3042B88BF0130FDF7DFFE32E768
:10353C0010A804F0D2FE3DE704F037FF3AE72D2047
:10354C00FDF782F849E706A804F0C7FE264B186879
:10355C00FDF7CCFE03A804F0C0FE1F4B186FFDF75F
:10356C00C5FE40E72D20FDF76FF84DE706A804F0E7
:10357C00B4FE1E4B1868FDF7B9FE03A804F0ADFEAF
:10358C00154BD3F88800FDF7B1FE43E72D20FDF76E
:10359C005BF850E706A804F0A0FE144B1868FDF782
:1035AC00A5FE03A804F099FE0B4BD3F8A000FDF781
:1035BC009DFE46E77C6800205C6800208468002043
:1035CC0080680020C8680020AC680020A868002033
:1035DC00C4680020A468002048320020006CDC0283
:1035EC00E0B1FFFF00389C1C6C680020686800206C
:1035FC0070B5BAB0A54B93E803003890ADF8E41061
:10360C00090C8DF8E610A24B93E803003690ADF848
:10361C00DC10090C8DF8DE109E4A33AB07CA03C3CD
:10362C0023F8022B120C1A709B4A30AB07CA83E8A2
:10363C0007009A4A2DAB07CA03C323F8022B120CBE
:10364C001A70974B29AC0FCB07C4238024AC954D33
:10365C000FCD0FC42B6823600DF1780C924C0FCC5E
:10366C00ACE80F0094E803004CF8040B8CF8001045
:10367C008E4B1AAC0FCB84E80F0015AC8C4D0FCDD4
:10368C000FC42B68236010AC8A4D0FCD0FC42B6870
:10369C0023800DF1280C884C0FCCACE80F0094E87B
:1036AC0003004CF8040B8CF8001005AC834D0FCDC7
:1036BC000FC42B682380824B0DF1040C0FCBACE8AC
:1036CC0007002CF8023B1B0C8CF800307D4B1B6860
:1036DC007D4A9342C0F093807C490A6842F0040210
:1036EC000A607B4A934204D2784A136843F004037D
:1036FC001360784B1B68B3B1774B186800EB400232
:10370C00D100764A4B1E13440F320A44002103F8B1
:10371C00011F9342FBD1714B00EB400203EBC20241
:10372C000021116151616B4B00221A606C4B1B68BC
:10373C007BB1144620266A4D3046FCF785FF0134D8
:10374C002B68A342F8D85E20FCF77EFF0D20FCF717
:10375C007BFF38A804F0C1FD5C4C206804F0E3FD4D
:10376C003D20FCF771FF236813F0010F69D1574B13
:10377C001B6813F0020F68D1544B1B6813F0040F35
:10378C0067D1524B1B6813F0080F66D14F4B1B6867
:10379C0013F0400F65D14D4B1B6813F0200F64D113
:1037AC004A4B1B6813F0800F63D1484B1B6813F412
:1037BC00807F62D1454B1B6813F4007F61D1434B72
:1037CC001B6813F4806F40F09380404B1B6813F41C
:1037DC00006F40F0918036A804F07FFD404B1868D4
:1037EC0004F0E7FB2920FCF72FFFFEF761FF0D200B
:1037FC00FCF72AFF3B4B00221A603AB070BD344AEA
:10380C009342FFF471AF314B1B68002B7FF471AF07
:10381C00304B1B68002B73D1334B1B68012BE6D04C
:10382C002020FCF711FF6F20FCF70EFF6B20FCF73C
:10383C000BFF2E4B1B68102BD9D14820FCF704FF33
:10384C00D5E733A804F049FD91E730A804F045FD15
:10385C0092E72DA804F041FD93E729A804F03DFD63
:10386C0094E724A804F039FD95E71EA804F035FD73
:10387C0096E71AA804F031FD97E710A804F02DFD87
:10388C0098E715A804F029FD99E700BF60810008AE
:10389C0068810008708100087C810008888100081C
:1038AC0094810008A4810008B8810008D081000828
:1038BC00E0810008F48100080882000820820008DA
:1038CC00348200089468002040670020D0680020F3
:1038DC005C660020D4680020B068002048320020CC
:1038EC0044680020E8680020D86800205C6800204C
:1038FC000AA804F0F2FC68E705A804F0EEFC6AE7FD
:08390C0001A804F0EAFC72E7D7
:1039140038B5FDF7FBFD0446002800F0D180C0B2A5
:103924006B4B1B683BB16B4B1B6823B16A4B187024
:103934006A4B01221A600A2800F0BF80022840F274
:10394400BE80644B1C684CB9092808BF2020644B16
:103954001B683F2B02D9202800F09A80282815D014
:103964002F283CD01B2863D1002C00F0A9800D2007
:10397400FCF76EFE5A4B1A685A4B20219954134493
:1039840000215970584B1A60022499E0574B1C6867
:103994000CB1002494E0FCF75BFEFDF7B7FD0028B2
:1039A400FBD0C0B220280BD04D490B684D4A2825C6
:1039B400D5541A44507002330B60FCF749FE7FE083
:1039C400474B1B680133494A13600820FCF740FE4B
:1039D4002020FCF73DFE0820FCF73AFE70E0434B44
:1039E4001C680CB100246BE0FCF732FEFDF78EFD81
:1039F4000028FBD0C0B22F280BD039490B68394AB4
:103A04002F25D5541A44507002330B60FCF720FE66
:103A140056E0334B1B680133344A13600820FCF72B
:103A240017FE2020FCF714FE0820FCF711FE47E0E7
:103A3400092847D0122847D0082818D12B4B1D68D5
:103A44000DB100243CE0264B1C68002C38D0631ECA
:103A5400234A13602024234AD454FCF7F9FD20465A
:103A6400FCF7F6FD0820FCF7F3FD2C4628E00D28B2
:103A740016D11B4B1B685BB9194B1A68194B2021D3
:103A84009954134400215970174B1A60012417E00C
:103A9400164B1B68012BEFD00D20FCF7D9FDEBE78B
:103AA400124B1C6894B90E4D2B680E4AD054FCF787
:103AB400CFFD2B6801332B6002E0002400E00024DA
:103AC400204638BD0324FBE70424F9E70024F7E784
:103AD40038020020CC6800201869002058680020B3
:103AE4004C6800205067002050680020D8680020EF
:103AF400164B1868164B1A5C202A0AD10344144941
:103B0400C1F10101C81813F8012F202AFAD00F4B74
:103B14001860AAB110B40F4901440F4C002311F8E6
:103B2400012F202A04D004F8012B0133102BF6D1E5
:103B3400094A0021D1540344084A136010BC704759
:103B4400054B00221A70054B18607047446800202A
:103B5400506700204F670020F46700204C68002065
:103B64002DE9F04F87B00F4601380DF10809494699
:103B7400002505E011F8013CFBB10135102D0CD0F6
:103B840010F8013F01F8013BA3F16102D2B2192AF6
:103B9400F0D8203B01F8013CEFE700238DF8173003
:103BA4009DF808302D2B0FD1264B00221A60012DD1
:103BB40042D9012301931E460EE000238DF81730ED
:103BC4009DF808302D2B29D01E4B00221A600120AD
:103BD4007DB3002301931E461A4BD3F8008006AB35
:103BE4001E44113E4FF0000A4FF0010B3446394693
:103BF40016F8010F04F0E9FBB0F1FF3F12D007FB08
:103C04000808DA460234A4EB0904AC42EED30D4BA7
:103C1400C3F80080019B7BB901200AE0012DC3D1C8
:103C2400002006E0BAF1000F02D0064BC3F8008072
:103C3400002007B0BDE8F08F024A13685B421360AE
:083C44000120F6E748680020AA
:103C4C0008B5364B187800285CD01A46002301338F
:103C5C0012F8011F0029FAD12D2811D030282DD1AE
:103C6C002E4A527802F0DF02582A15D02C4A1168DD
:103C7C0010290DD02D283BD00A2B47D900204BE022
:103C8C00012B39D0264A1168102931D12D282BD07F
:103C9C00082B3BD900203FE0204A92782D2A09D0EE
:103CAC000A2B2BD810211F48FFF756FF003818BFDE
:103CBC00012031E00B2BF5D900202DE02528D5D1A2
:103CCC00164A52782D2A09D00B2B19D80A211648DE
:103CDC00FFF742FF003818BF01201DE00C2BF5D96F
:103CEC00002019E00023D1E7092B0FD9002013E0A5
:103CFC000B2B0BD900200FE000200DE000200BE077
:103D0C00002009E0064B19681029EBD00348FFF797
:103D1C0023FF003818BF012008BD00BFF467002046
:0C3D2C005C680020F6670020F5670020AE
:103D380070B41B4D00241B4E06F1FF3C284610F8BA
:103D4800013B1CF8012FA3F16101C9B219290BD855
:103D5800203BDBB2A2F16101C9B219290CD8203A83
:103D6800D2B29A42EBD014E0A2F16101C9B219298A
:103D78000BD9202B08BF002393420AD1002ADED199
:103D8800094B1C60012070BC7047203AD2B2202B2E
:103D9800E7D1013408358D2CCED10020F3E700BFE0
:0C3DA8003C790008F4670020A0680020AF
:103DB4001D4B1B788BB330B51B4A00231C460133C3
:103DC40012F8181F0029F9D1B4F1FF3F27D004EBF2
:103DD4004405154B03EBC505013D08E0134B1C607E
:103DE400012030BD013C183DB4F1FF3F19D010490A
:103DF40001F1100EAC461CF8010F11F8013BA3F1C0
:103E04006102D2B2192A9CBF203BDBB28342E9D1C2
:103E14000028E3D07145EED1E4E70020704700208C
:103E2400DFE70020DDE700BF48320020A068002063
:043E3400F46700200F
:103E380008B52A4B1A682A4B1A60FFF757FEFFF796
:103E4800B5FF00283ED0254B1A68254B1A60254B34
:103E58001B68062B3CD9244A1360244903EB430210
:103E6800D00001EBC2024FF0000C01F800C052690B
:103E7800C2F30B021E4802601E48026003EB4303B4
:103E880001EBC30301F57C618B420AD20139C91ADF
:103E980021F0030104311944604643F8040B8B42B6
:103EA800FBD140F6FE339A420BD89300043B124AEA
:103EB800134402F53F523832002143F8041F93425D
:103EC800FBD108BD0D4A136843F021031360F8E7DE
:103ED8000A4A136843F080031360F2E74C68002035
:103EE80044680020A0680020B06800204832002004
:103EF800E0680020DC68002048020020D06800202C
:103F080008B50E4B1A680E4B1A60FFF7EFFDFFF766
:103F18004DFF28B10B4B1B6801330B4A136008BDDA
:103F28000A4B1B78302B05D0094A136843F021034C
:103F38001360F4E7044B00221A60F0E74C68002095
:103F480044680020A0680020F0680020F467002082
:043F5800D06800200D
:103F5C00084A1368084941F823000133136040F6FE
:103F6C00FE32934204D9054A136843F020031360D0
:103F7C00704700BFE068002048020020D068002095
:103F8C0008B5154B1868154B53F8203013F4002F57
:103F9C000AD1134A12689AB913F4003F0AD1114B93
:103FAC0053F82030984704E00F4A136843F4007329
:103FBC00136008BD0C4A136843F008031360F8E75C
:103FCC0013F4803F04D0074B53F820309847F0E7A8
:103FDC00FFF7BEFFEDE700BFA068002008770008E0
:0C3FEC00D468002000000020D0680020F5
:103FF800F0B595B00CAC3D4D0FCD0FC495E80F0052
:1040080084E80F0005AC3A4D0FCD0FC495E80700C2
:1040180003C422706C46374D0FCD0FC42B68237034
:10402800354B1B68522B0DD9344D334FA5F1510632
:104038002C4615F8010FFCF709FB0234A41B3B685A
:10404800A342F5D852232E4A13602E4A13602C4CF3
:104058002D4E02E022682B4B1A60274D22682B68F0
:104068009A4231D2FFF742FD3378002BF6D0FFF7A2
:10407800E9FD58B1254B1A68254B1A60254B1B687A
:10408800002BE7D0244B01221A60E3E7FFF750FE2C
:1040980080B1224B1A68224B53F8223013F4802F38
:1040A8001FD0FFF76FFF1F4B1B683BB92268154BEA
:1040B8001A60D2E70CA804F012F905E0194B0022A7
:1040C8001A60684604F00BF90D20FCF7BFFA52237A
:1040D800094A13600A4A1360134B00221A6015B08C
:1040E800F0BD05A804F0FBF8EEE700BFF87F000874
:1040F800188000083480000850680020A16700205C
:104108004C68002044680020F467002048680020BC
:10411800E4680020CC680020E8680020A06800203F
:0C41280008770008D0680020D86800204C
:1041340010B5294B1A68294B1A60FFF7D9FCFFF711
:1041440037FE00282DD0244B1A68244B1A60244BC8
:104154001B6803EB4301234A02EBC102526912F0CC
:10416400406F24D0204A126862B1204A12684AB1D2
:104174001E4A002111601E490A68101D08601D496D
:10418400096851601C4A1268BAB91948026852F8A1
:10419400044903EB4303134901EBC3031C610260AD
:1041A40004E0164A136843F0A003136010BD134AD9
:1041B400136843F080031360F8E77B20FFF7CCFE1D
:1041C400074B186800EB4000064B03EBC0001030AF
:1041D400FFF7C2FEEAE700BF4C68002044680020F5
:1041E400A068002048320020CC680020E868002045
:1041F40094680020E4680020D4680020D06800207F
:1042040008B57C20FFF7A8FE054A1368191D116044
:10421400044A12685A604FF0FF30FFF79DFE08BD54
:0842240094680020E06800200E
:10422C0008B57D20FFF794FE054A1368191D11602F
:10423C00044A12685A604FF0FF30FFF789FE08BD40
:08424C0094680020E0680020E6
:1042540008B57E20FFF780FE054A1368191D11601A
:10426400044A12685A604FF0FF30FFF775FE08BD2C
:0842740094680020E0680020BE
:10427C0008B57F20FFF76CFE054A1368191D116005
:10428C00044A12685A604FF0FF30FFF761FE08BD18
:08429C0094680020E068002096
:1042A40038B58020FFF758FE094C25684FF0FF30E1
:1042B400FFF752FE074B1A6810680749236803F199
:1042C4008043013B01EB830341F82030156038BD86
:0C42D400E06800209468002048020020F0
:1042E00008B58120FFF73AFE054A1368191D1160D1
:1042F000044A12685A604FF0FF30FFF72FFE08BDE6
:0843000094680020E068002031
:1043080038B58220FFF726FE0C4C236818680C4D40
:1043180005EB8000FFF71EFE23681A68094B1B682F
:1043280003F18043013B05EB830345F822308720E6
:10433800FFF710FE2368043B236038BD9468002013
:0843480048020020E06800209B
:1043500038B58320FFF702FE0C4C236818680C4D1B
:1043600005EB8000FFF7FAFD23681A68094B1B680C
:1043700003F18043013B05EB830345F8223087209E
:10438000FFF7ECFD2368043B236038BD94680020F0
:0843900048020020E068002053
:1043980038B58420FFF7DEFD0C4C236818680C4DF7
:1043A80005EB8000FFF7D6FD23681A68094B1B68E8
:1043B80003F18043013B05EB830345F82230872056
:1043C800FFF7C8FD2368043B236038BD94680020CC
:0843D80048020020E06800200B
:1043E00008B58520FFF7BAFD054A1368191D11604D
:1043F000044A12685A604FF0FF30FFF7AFFD08BD66
:0844000094680020E068002030
:1044080038B58620FFF7A6FD0C4C236818680C4DBC
:1044180005EB8000FFF79EFD23681A68094B1B68AF
:1044280003F18043013B05EB830345F822308820E4
:10443800FFF790FD2368043B236038BD9468002093
:0844480048020020E06800209A
:1044500008B5234B1B68BBB9224B1B681968224A5D
:104460001160224A934230D9214A1268022A1FD091
:10447000043B1C4A13601F4A1368013B13601E4B28
:104480001A681E4B1A6008BD7720FFF767FD0022EF
:10449000134B1A601A490B6801330B6003EB43039B
:1044A000DB001849CA54184B1A68184B1A60E6E723
:1044B000104A1168164A12689142D9D1144A002153
:1044C00011600B4A03211160D2E7074B00221A60EA
:1044D000074B1B68022BD2D1054B03221A60CEE793
:1044E000D46800209C680020C0680020506500202F
:1044F00038020020B4680020340200205C680020EC
:10450000B068002048320020E0680020DC6800200D
:04451000EC68002033
:1045140038B5324B1B684BBB314B1B681C6824F409
:104524000024A4F17203022B16D97D20FCF790F825
:104534002020FCF78DF8FEF785FBA4F18105072DFB
:1045440015D9853C012C1CD9032D0FD8254B1B688C
:10455400188803F0ECFE09E0234B18680430C0F31C
:104564000B0003F0E4FE2920FCF772F838BD20208C
:10457400FCF76EF85220FCF76BF83A20FCF768F869
:10458400DFE7184B1A68194BD31A082BEED932F807
:104594000C0C03F0CCFE2020FCF75AF82020FCF78A
:1045A40057F8104C236833F8080C03F0C0FE2020A1
:1045B400FCF74EF86920FCF74BF8236833F8040C39
:1045C40003F0B5FE2020FCF743F87820FCF740F810
:1045D40023681888043003F0AAFEC7E7D0680020D7
:1045E400BC6800209C680020C06800205065002042
:1045F40070B5444B002103F57C6243F8041B9342DD
:10460400FBD1414B03F54051002243F8042F8B4268
:10461400FBD100233D4A13600A223D490A603D490B
:104624000A603D4A13603D4A012111603C4A13600F
:104634003C4A082111603C4A322111603B4A136014
:104644004FF0FF323A490A603A490A603A490B602E
:104654003A4B1A602B4B31224FF0560C00214FF08D
:10466400406083F800C05A7099705861196118331A
:104674000132D2B2352AF4D1224B4E2583F8605050
:10468400532483F861404FF0540E83F862E04FF0F6
:10469400500C83F863C0312283F86420002283F82D
:1046A40065204FF0406058674FF0FF31196783F879
:1046B400785083F8794083F87AE083F87BC0322617
:1046C40083F87C6083F87D20C3F88C00C3F88810DD
:1046D40083F8905083F8914083F892E083F893C074
:1046E400332483F8944083F89520C3F8A400C3F8D6
:1046F400A010134B1A60134B07221A60FDF7DCFF5E
:1047040070BD00BF48320020440200200C69002024
:10471400340200205C680020F06800203802002089
:104724007C6800208468002080680020C86800201D
:10473400AC680020A8680020C4680020A468002099
:08474400E0680020B0680020CD
:10474C00064B1868064B1B68984205D032BF181AE6
:10475C00C01A00F58060704700207047FC6800208C
:04476C0000690020C0
:1047700010B5084B1C68221D1A60074B1B682BB133
:10478000064B1B6813B1064B186801E0FFF7DEFF0C
:10479000606010BD9468002038020020CC680020C2
:0447A0005868002035
:1047A40010B40C4B1C680C4921440C48002311F82C
:1047B400012F202A04D000F8012B0133502BF6D10D
:1047C400064A0021D1542344054A1360012010BC39
:1047D400704700BF446800204F670020F467002042
:0447E4004C680020FD
:1047E8002DE9F843834B1B680133834A1360FFF7B5
:1047F800D5FF824A0026344603E001360134502CA6
:104808000DD012F8013B5C2BF7D0222BF6D17B4B55
:1048180000221A557A4B1D6845B9784CA3E0794AAD
:10482800136843F002031360BDE8F8837820FFF7AC
:1048380091FB754B1D68A4EB4604744A42F8254069
:1048480001351D6000263046324633466B4C6F4FAB
:104858004FF0010C03E00133E15C00296ED0E15C0C
:104868005C290BD0914008430832182AF3D947F83D
:1048780025000135664600200246ECE7E11891F86C
:1048880001E003F10209AEF16101192904D8AEF182
:10489800200EAEF1370807E0BEF12F0F13D9AEF1A5
:1048A8003008B8F1090FF4D8B8F10F0F14D814F87C
:1048B80009E00333AEF16101192916D8AEF1200ED3
:1048C800AEF1370118E00EB14F4B1D604D4A136829
:1048D80043F002031360A7E70EB14B4B1D60494A32
:1048E800136843F0020313609EE7BEF12F0F13D93C
:1048F800AEF130010929E3D80F2916D801EB0811C8
:10490800914008430832182AA6D947F825000135EE
:104918006646002002469FE70EB13B4B1D60394AB0
:10492800136843F0020313607EE70EB1364B1D6037
:10493800344A136843F00203136075E70EB1324B33
:104948001D60002A3FF470AF2F4A13682F4941F8C1
:1049580023000133136067E7FBF778FE0135635DD9
:10496800002B3FF461AF605D5C28F5D163195B787B
:10497800A3F16102192A03D8203BA3F1370205E00D
:104988002F2B10D9A3F13002092AF6D80F2A10D8F4
:1049980063199B780335A3F1610119290FD8203BCE
:1049A800A3F1370011E0174A136843F002031360BC
:1049B8003AE7144A136843F00203136034E72F2BD5
:1049C8000BD9A3F130000928EAD80F280BD800EB3F
:1049D8000210C0B2FBF73AFEC1E70A4A136843F077
:1049E8000203136020E7074A136843F002031360C9
:1049F8001AE700BF4C68002044680020F4670020D4
:104A0800D4680020D0680020E06800204802002018
:104A1800374B1B68B3F5803F35D3354B4FF6FF72E4
:104A28001A60344B1B6813F0010F12D1314B00226E
:104A38001A611A6030498A6D42F002028A6546F2AC
:104A480060029A614FF4FA62DA621A6842F001026F
:104A58001A60274B1B68013B264A9362274B1B6849
:104A6800002B40DB234A136A43F001031362244BF3
:104A78001B68002B1F4A136AB4BF23F0100343F0CE
:104A8800100313627047002BCBD11A4A136823F026
:104A9800010313604FF0FF30184B18604FF090433C
:104AA800196821F440511960D96821F44051D9603E
:104AB800D96841F40051D960116A21F001011162ED
:104AC8000F490860196821F440411960D96821F438
:104AD8004041D960D96841F40041D960136A23F094
:104AE800100313627047136A23F001031362BEE7D1
:104AF800C86800200004004000100240AC68002094
:044B0800A868002079
:104B0C004FF09042136823F440531360224A136A07
:104B1C0023F001031362214B1B68002B20DB4FF0A9
:104B2C009041CA6822F44052CA6003B3B3F5FA6FDD
:104B3C0025DA4FF090431A6842F400521A601A6A50
:104B4C0022F070621A621A6A42F000721A62124BF8
:104B5C001A6A42F001021A62104A12685A637047CC
:104B6C004FF09042D36843F40053D36070470A6807
:104B7C0042F480520A604FF480028A617047074BFE
:104B8C004FF4FA621A604FF090431A6842F4805264
:104B9C001A6040229A61704700040040AC68002003
:104BAC0008B5124B1B6863B1114B1B684BB1104B12
:104BBC0000221A600F4A1368191D11600E4A126800
:104BCC005A600C4A136853F804090C4908601360C6
:104BDC000B4B1B6813F0010F02D0FFF791FF08BDC0
:104BEC00084B18221A60FFF711FFF6E7CC6800207B
:104BFC00E868002094680020E4680020AC6800207D
:084C0C0000040040C86800200C
:104C14004FF09042136823F440431360224A136A0E
:104C240023F010031362214B1B68002B20DB4FF091
:104C34009041CA6822F44042CA6003B3B3F5FA6FE4
:104C440025DA4FF090431A6842F400421A601A6A57
:104C540022F070421A621A6A42F000521A62124B2F
:104C64001A6A42F010021A62104A12689A63704774
:104C74004FF09042D36843F40043D36070470A680E
:104C840042F480420A604FF400028A617047074B85
:104C94004FF4FA621A604FF090431A6842F480426B
:104CA4001A6080229A61704700040040A8680020BE
:104CB40008B50F4B1B6863B10E4B1B684BB10D4B12
:104CC40000221A600C4A1368191D11600B4A1268FD
:104CD4005A60094A136853F80409094908601360C3
:104CE400FFF798FEFFF710FFFFF792FF08BD00BF24
:104CF400CC680020E868002094680020E468002064
:044D0400C86800205B
:104D080008B5124B1B6863B1114B1B684BB1104BB4
:104D180000221A600F4A1368191D11600E4A1268A2
:104D28005A600C4A136853F804090C490860136068
:104D38000B4B1B6813F0010F02D0FFF767FF08BD8C
:104D4800084B18221A60FFF763FEF6E7CC680020CC
:104D5800E868002094680020E4680020A868002023
:084D680000040040C8680020AF
:104D70002C4B1B68B3F5803F2ED32A4B4FF6FF72A6
:104D80001A604FF080431B6813F0010F13D14FF0EE
:104D9000804300221A611A6023498A6D42F00102A1
:104DA0008A6546F260029A614FF4FA62DA621A6822
:104DB00042F001021A601B4B1B68013B4FF080421E
:104DC00093621A4B1B68002B24DB4FF08042136A5E
:104DD00043F0100313627047002BD2D14FF0804292
:104DE000136823F001031360104B4FF0FF3119607B
:104DF0000F4B196821F0C0011960D96821F0C0017A
:104E0000D960D96841F08001D960136A23F010039A
:104E10001362704702F58062136A23F01003136275
:104E2000704700BFC468002000100240A468002042
:044E30000004004832
:104E3400244A136823F0C00313604FF08042136ABE
:104E440023F010031362204B1B68002B1FDB1D494A
:104E5400CA6822F0C002CA60FBB1B3F5FA6F24DA63
:104E6400184B1A6842F080021A601A6A22F47042DF
:104E74001A621A6A42F480521A624FF080431A6A24
:104E840042F010021A62104A12689A6370470D4A7F
:104E9400D36843F08003D36070470A6842F040024D
:104EA4000A604FF400228A617047074B4FF4FA629C
:104EB4001A60044B1A6842F040021A6008229A6190
:0C4EC400704700BF00040048A4680020F4
:104ED00008B50E4B1B6863B10D4B1B684BB10C4BF7
:104EE00000221A600B4A1368191D11600A4A1268E1
:104EF0005A60084A136853F80409084908601360A7
:104F0000FFF736FFFFF796FF08BD00BFCC68002013
:104F1000E868002094680020E4680020C46800204D
:104F200008B5134B1B6863B1124B1B684BB1114B97
:104F300000221A60104A1368191D11600F4A126886
:104F40005A600D4A136853F804090D49086013604C
:104F50004FF080431B6813F0010F02D0FFF76AFF88
:104F600008BD084B18221A60FFF702FFF6E700BFE2
:104F7000CC680020E868002094680020E4680020E5
:084F8000A4680020C4680020B1
:104F8800074A136853F804091360322807D99F2881
:104F980004D8044A136843F480631360A038704748
:084FA80094680020D06800208D
:104FB00008B5FFF7E9FF174B1B687BB9430003F007
:104FC0001E030F280BD84FF090421269134012496C
:104FD0000A68101D0860D3B10123536008BD1F2863
:104FE00003D80E4A12691340F1E72F2803D80C4A60
:104FF00012691340EBE7322804D0064B4FF480626D
:105000001A60EBE7074B1B6903F00403DFE700239B
:105010005360E3E7D0680020946800200004004853
:0850200000080048000C0048E4
:10502800042807D005281CD1174A136823F48033B5
:1050380013607047144A136823F001031360134B7D
:105048001B68B3F1FF3F0BD0072809D14FF080420E
:10505800136A23F0100313620C4B4FF0FF321A60EF
:1050680070470B4B1B68B3F1FF3FE8D00628E6D129
:105078004FF08042136A23F001031362044B4FF090
:10508800FF321A60704700BF00080050A86800206F
:04509800AC680020E0
:10509C0010B5FFF773FF474B1B685BB904460F282D
:1050AC0021D8831E012B01D9052804D1414B4FF483
:1050BC0080621A6010BDFFF7B1FF620003219140BE
:1050CC004FF09043D86820EA0100D860186820EAB5
:1050DC00010119601868012101FA02F202431A60F9
:1050EC00A1409961E6E71F281CD92F284AD8A0F1C6
:1050FC00200C2D2841D04FEA4C02032090402E4B1F
:10510C00DC6824EA0004DC601C6824EA00001860F7
:10511C001868012101FA02F202431A6001FA0CF13B
:10512C009961C7E7A0F11004244B1B68B3F1FF3F52
:10513C0001D0032C16D062004FF0030C0CFA02FCC9
:10514C001F4BD86820EA0C00D860186820EA0C00C5
:10515C0018601868012101FA02F202431A60A1409A
:10516C009961A7E74FF08042136A23F001031362A1
:10517C00124B4FF0FF321A60DDE70E4B4FF480629A
:10518C001A6097E7322804D00A4B4FF480621A60F9
:10519C0090E70C4BDA6822F03002DA601A6822F0E1
:1051AC0030021A601A6842F010021A6004229A61E6
:1051BC0080E700BFD068002000080048A4680020E9
:0851CC0000040048000C00483B
:1051D40010B5FFF7D7FE464B1B685BB904460F2892
:1051E40022D8831E012B01D9052804D1404B4FF44A
:1051F40080621A6010BDFFF715FF62000321914021
:105204004FF09043D86820EA0100D860186820EA7B
:10521400010119601868012101FA02F202431A60BF
:105224001034A1409961E5E71F281BD92F2847D8DE
:10523400A0F120032D283ED05B00032199402D4A84
:10524400D06820EA0100D060106820EA01011160F2
:105254001068012101FA03F303431360103CA140D9
:105264009161C7E7A0F11003234A1268B2F1FF3F2E
:1052740001D0032B14D05B00032199401F4AD0684E
:1052840020EA0100D060106820EA01011160106872
:10529400012101FA03F303431360A1409161A9E7DB
:1052A4004FF080410A6A22F001020A62124A4FF06A
:1052B400FF311160DFE70E4B4FF480621A6099E70B
:1052C400322804D00A4B4FF480621A6092E70C4BE8
:1052D400DA6822F03002DA601A6822F030021A60CA
:1052E4001A6842F010021A604FF480229A6181E732
:1052F400D068002000080048A4680020000400488A
:04530400000C004851
:1053080010B5FFF73DFE404B1B685BB904460F28FC
:105318001FD8831E012B01D9052804D13A4B4FF41D
:1053280080621A6010BDFFF77BFE64000322A24072
:105338004FF09043196821EA02011960D96821EAFF
:105348000202DA60D968012202FA04F40C43DC6034
:10535800E8E71F2817D92F2841D8A0F120022D28C7
:1053680038D0510003228A40284B186820EA0200EE
:105378001860D86820EA0202DA60D86801228A40F8
:105388000243DA60CEE7A0F11004214B1B68B3F1A9
:10539800FF3F01D0032C12D064000322A2401D4B12
:1053A800196821EA02011960D96821EA0202DA6063
:1053B800D968012202FA04F40C43DC60B2E74FF02A
:1053C8008042136A23F001031362114B4FF0FF323E
:1053D8001A60E1E70C4B4FF480621A60A2E73228AA
:1053E80004D0094B4FF480621A609BE70A4BDA68D5
:1053F80022F03002DA601A6822F030021A60DA68A5
:1054080042F01002DA608DE7D068002000080048FA
:0C541800A468002000040048000C0048BC
:1054240010B5FFF7AFFD404B1B685BB904460F286E
:105434001FD8831E012B01D9052804D13A4B4FF400
:1054440080621A6010BDFFF7EDFD64000322A240E4
:105454004FF09043196821EA02011960D96821EAE2
:105464000202DA60D968022202FA04F40C43DC6016
:10547400E8E71F2817D92F2841D8A0F120022D28AA
:1054840038D0510003228A40284B186820EA0200D1
:105494001860D86820EA0202DA60D86802228A40DA
:1054A4000243DA60CEE7A0F11004214B1B68B3F18C
:1054B400FF3F01D0032C12D064000322A2401D4BF5
:1054C400196821EA02011960D96821EA0202DA6046
:1054D400D968022202FA04F40C43DC60B2E74FF00C
:1054E4008042136A23F001031362114B4FF0FF3221
:1054F4001A60E1E70C4B4FF480621A60A2E732288D
:1055040004D0094B4FF480621A609BE70A4BDA68B7
:1055140022F03002DA601A6822F030021A60DA6887
:1055240042F02002DA608DE7D068002000080048CD
:0C553400A468002000040048000C00489F
:1055400010B5FFF721FD374B1B685BB904460F28E8
:105550001AD8831E012B01D9052804D1314B4FF4F1
:1055600080621A6010BDFFF75FFD6400032303FA39
:1055700004F44FF090431A6822EA04021A60DA68D1
:1055800022EA0404DC60EDE71F2812D92F2837D85F
:10559000A0F120022D282ED0530003229A40224B46
:1055A000196821EA02011960D96821EA0202DA6069
:1055B000D8E7A0F110041D4B1B68B3F1FF3F01D0E9
:1055C000032C0DD06400032303FA04F4184B1A686B
:1055D00022EA04021A60DA6822EA0404DC60C1E705
:1055E0004FF08042136A23F0010313620F4B4FF018
:1055F000FF321A60E6E70B4B4FF480621A60B1E7A6
:10560000322804D0074B4FF480621A60AAE7094B96
:105610001A6822F030021A60DA6822F03002DA608A
:10562000A0E700BFD068002000080048A468002060
:0856300000040048000C0048D2
:1056380038B5414BDB6C13F4005F00D038BD3E4BEE
:10564800DA6A22F40052DA62DA6C42F40052DA645E
:105658004FF0A044A36823F00053A360A36843F06D
:105668008053A360354DAB6823F00053AB60AB6843
:1056780043F08053AB600220FAF7D8FED4F8B0307C
:1056880023F47F4323F0FE03C4F8B030D5F8B030DC
:1056980023F47F4323F0FE03C5F8B030284B4FF4C2
:1056A80040329A60FAF79AFE236843F001032360B8
:1056B800A36843F00103A3602246136813F0010FA7
:1056C800FBD04FF0A0431A6842F001021A604FF075
:1056D8000042DA601B4A5A6102F160429A6103F59E
:1056E80080731A6842F001021A609A6842F0010257
:1056F8009A601A46136813F0010FFBD00F4B1A6813
:1057080042F001021A604FF00042DA600D4A5A6115
:1057180002F160429A614FF0A04100220A634A6395
:105728008A63CA631A635A639A63DA63FAF756FE9E
:10573800FAF754FE82E700BF001002400001005053
:085748000003005024499224E3
:105750004FF0A0431A6842F001021A609A6842F0C2
:1057600002029A6003F580731A6842F001021A601F
:105770009A6842F002029A604FF0A042936813F0D8
:10578000010FFBD1044BDA6C22F40052DA64DA6ABE
:0C57900042F40052DA6270470010024040
:10579C0010B58AB00DF1100C9D4C0FCCACE80F007D
:1057AC0094E803004CF8040B8CF80010994B6C46F1
:1057BC000FCB07C42370984B1B681C68B4F1FF3FD8
:1057CC0036D0964BDB6C13F4005F3AD04FF0A0430D
:1057DC0040F2FF721A6004F0A003A02B37D06300D4
:1057EC0003F01E03032202FA03F3072C46D9A4F19B
:1057FC00B002152A00F23681B03C152C00F2328131
:10580C00DFE814F0CA00D40030013001300130015F
:10581C0030013001300130013001300130013001F4
:10582C0030013001DE00E800F200FC001C01260112
:10583C00043B794A1360FFF785FF684602F04DFD83
:10584C003BE0FFF7F3FE04A802F047FDBEE704F0CF
:10585C000F025300032101FA03F314F0080F40F078
:10586C000181072A00F2FE80DFE812F00A0029000D
:10587C00FC00FC003400540064007D002246F0E77C
:10588C004FF09042116819431160D16821EA03036B
:10589C00D360012292014FF0A0431A639A6842F040
:1058AC0004029A601A46136813F0080FFBD05A4B87
:1058BC001B684FF0A042126C1A600AB010BD4FF07A
:1058CC009042116819431160D16821EA0303D36037
:1058DC000222DFE752490A6822F001020A604FF007
:1058EC009042116819431160D16821EA0303D36017
:1058FC0011239B014B4A1363936843F00403936099
:10590C00136813F0080FFBD0434B1B68454A126C0D
:10591C001A60D2E742490A6822F480320A604FF0DA
:10592C009042116819431160D16821EA0303D360D6
:10593C000D23DEE73C4A1268B2F1FF3F08D03B4929
:10594C000A6A22F001020A62374A4FF0FF311160F5
:10595C004FF09042116819431160D16821EA03039A
:10596C00D3600323C5E7324A1268B2F1FF3F08D077
:10597C002E490A6A22F010020A622D4A4FF0FF31BA
:10598C0011604FF09042116819431160D16821EAFF
:10599C000303D3600423ACE7264A11681943116052
:1059AC00D16821EA0303D3600F23A2E7214A1168CF
:1059BC0019431160D16821EA0303D3600C2398E7E3
:1059CC001D4A116819431160D16821EA0303D360A1
:1059DC0006238EE7184A116819431160D16821EA31
:1059EC000303D360072384E7134A1168194311603A
:1059FC00D16821EA0303D36008237AE70E4A1168C1
:105A0C0019431160D16821EA0303D360092370E7BD
:105A1C00448200085C820008946800200010024058
:105A2C000008005000010050AC6800200004004049
:105A3C00A868002000040048000800480C4A1168BF
:105A4C0019431160D16821EA0303D360052350E7A1
:105A5C00074A116819431160D16821EA0303D36026
:105A6C000B2346E7034A136843F48063136024E76F
:085A7C0000080048D06800207A
:105A8400174B1B68032B24D8164B1B68043B1C2B99
:105A94001FD8154B1B68B3F5803F1AD2134B1A68F5
:105AA40022F47C621A601A6842F488621A60DA6826
:105AB40022F44072DA60DA6842F40072DA60084B69
:105AC4001B68012B094B8CBF08224FF400229A61FA
:105AD4007047074A136843F480631360704700BF3C
:105AE4007C6800208468002080680020000400484E
:045AF400D068002056
:105AF80010B50C4A1368194651F804490A4804605D
:105B0800116053F8040C09490860A3F108011160F9
:105B180053F8080C064908600C3B1360FFF7AEFF0A
:105B280010BD00BF946800208068002084680020B1
:045B38007C68002065
:105B3C002DE9F0479E4B1B6803F4A863B3F5886FFF
:105B4C002BD19C4B1B681D689B4B1A689B4B1C688C
:105B5C00002C5BD1964B4FF400219961984B18683F
:105B6C00F0B90127924B4FF4001E4FF0200C0E465B
:105B7C000824013A07FA02F1294214BFC3F818C0ED
:105B8C00C3F818E09E611969C1F3001141EA4000A5
:105B9C009C61002AEDD104462FE0FFF76DFFD0E7A2
:105BAC004FF00108824E4FF4001A4FF020094FF4C9
:105BBC00002E834F83484AF6AA214FF0080C013A75
:105BCC0008FA02F32B4214BFC6F81890C6F818A0B6
:105BDC00C6F818E03B6813B10160013BFCD1336996
:105BEC00C3F3001343EA4404C6F818C03B6813B16E
:105BFC000160013BFCD1002AE1D16D4B4FF4002236
:105C0C009A616C4B1B681C60BDE8F087012C25D099
:105C1C00022C78D0664B08219961694B1C68002CCA
:105C2C0040F0D2800127624B4FF4001E4FF0200C45
:105C3C004FF400260846013A07FA02F1294214BF34
:105C4C00C3F818C0C3F818E09E611969C1F30011BC
:105C5C0041EA44049861002AEDD1E3E0544B4FF43F
:105C6C0000219961564B1C68D4B90127504B4FF455
:105C7C00001E4FF0200C08260846013A07FA02F1E4
:105C8C00294214BFC3F818C0C3F818E09E61196903
:105C9C00C1F3001141EA44049861002AEDD12DE0D2
:105CAC0000244FF00108424E4FF4001A4FF0200927
:105CBC004FF0080E424F43484AF6AA214FF4002CED
:105CCC00013A08FA02F32B4214BFC6F81890C6F832
:105CDC0018A0C6F818E03B6813B10160013BFCD179
:105CEC003369C3F3001343EA4404C6F818C03B6895
:105CFC0013B10160013BFCD1002AE1D12C4B4FF4D4
:105D0C0000229A617DE72A4B082199612C4B1C6873
:105D1C00DCB90127264B4FF4001E4FF0200C0E4629
:105D2C004FF40020013A07FA02F1294214BFC3F8DC
:105D3C0018C0C3F818E09E611969C1F3001141EA5B
:105D4C0044049861002AEDD12DE000244FF00108A5
:105D5C00174E4FF4001A4FF020094FF0080E184F51
:105D6C0018484AF6AA214FF4002C013A08FA02F31B
:105D7C002B4214BFC6F81890C6F818A0C6F818E045
:105D8C003B6813B10160013BFCD13369C3F30013D1
:105D9C0043EA4404C6F818C03B6813B10160013BE8
:105DAC00FCD1002AE1D1024B08229A6129E700BFFD
:105DBC000004004894680020846800207C6800205F
:105DCC00806800200030004000244FF00108174E7E
:105DDC004FF4001A4FF020094FF4002E144F1548C1
:105DEC004AF6AA214FF0080C013A08FA02F32B42AA
:105DFC0014BFC6F81890C6F818A0C6F818E03B688F
:105E0C0013B10160013BFCD13369C3F3001343EAC6
:105E1C004404C6F818C03B6813B10160013BFCD1C7
:105E2C00002AE1D1014B08229A61EAE600040048FD
:085E3C008068002000300040E6
:105E4400304B1B6F002B5BDD2F4A1268002A2CDBC2
:105E54002E490A602E4A1268032A4AD8DFE802F063
:105E6400020F14194FF090424FF4803191614FF4B6
:105E74000031916126490A6801320A6011E04FF04D
:105E8400904202219161F5E74FF090420121916126
:105E9400F0E74FF090424FF4003191611C4A002129
:105EA4001160013B174A13677047524217490A6051
:105EB400174A1268032A1CD8DFE802F0020B1015F7
:105EC4004FF090424FF4803191614FF40031916171
:105ED400D0E74FF0904201219161CBE74FF090421F
:105EE40002219161C6E74FF090424FF480319161F5
:105EF400D4E707490A6801320A60032ACEDCD0E7F6
:105F0400704700BF483200206C6800209068002071
:045F14007868002089
:105F180008B5384B1B6863B1374B1B684BB1364B20
:105F280000221A60354A1368191D1160344A126834
:105F38005A60344B1B6FB3F1FF3F29D0324B1B68BB
:105F48006BB9324A1360324A13604FF090431A68B3
:105F580022F00F021A601A6842F005021A602749F7
:105F68000B6853F80429284802600B6052B94FF0B7
:105F780090434FF480329A614FF400329A61214B7A
:105F880000221A67224B00221A60FFF757FF08BD4C
:105F98001D4B00221A604FF090431A6822F00F023E
:105FA8001A601A6842F005021A60144B1A681368DE
:105FB800002B09DD4FF090434FF480329A610222A2
:105FC8009A61FEF7EFFDE2E7002B08DB4FF0904304
:105FD8004FF480329A614FF400329A61F1E75B42E4
:105FE80013604FF0904301229A614FF400329A6196
:105FF800E7E700BFCC680020E8680020946800202C
:10600800E4680020483200206C680020786800208E
:04601800906800206C
:10601C002F4BD3F88830002B58DD2E4A1268002AFB
:10602C002BDB2D490A602D4A1268032A47D8DFE87A
:10603C0002F00212171C2A4A4FF0807191614FF046
:10604C000071916125490A6801320A60013B204ABE
:10605C00C2F888307047224A4FF400719161F1E721
:10606C001F4A4FF480719161ECE71D4A4FF00071AB
:10607C0091611A4A00211160E8E7524216490A6000
:10608C00164A1268032A1AD8DFE802F0020A0F1423
:10609C00134A4FF0807191614FF000719161D1E71B
:1060AC000F4A4FF480719161CCE70D4A4FF40071A7
:1060BC009161C7E70A4A4FF080719161D9E70749AE
:1060CC000A6801320A60042AD3D0BFE7704700BFC8
:1060DC0048320020686800208C680020746800201A
:0460EC000004004864
:1060F00008B5374B1B6863B1364B1B684BB1354B4A
:1061000000221A60344A1368191D1160334A12685C
:106110005A60334BD3F88830B3F1FF3F28D0314B6E
:106120001B6863B9304A1360304A1360304B1A68F9
:1061300022F470221A601A6842F4A0221A602649DA
:106140000B6853F80429274802600B6052B9284BAA
:106150004FF080729A614FF000729A61204B0022DA
:10616000C3F88820214B00221A60FFF757FF08BDB3
:106170001C4B00221A601E4B1A6822F470321A60FF
:106180001A6842F4A0321A60134B1A681368002B85
:1061900009DD174B4FF080729A614FF400729A61DB
:1061A000FEF7B2FDE3E7002B07DB114B4FF08072E7
:1061B0009A614FF000729A61F2E75B4213600C4BF8
:1061C0004FF480729A614FF000729A61E8E700BF65
:1061D000CC680020E868002094680020E468002073
:1061E0004832002068680020746800208C68002015
:0461F000000400485F
:1061F400324BD3F8A030002B5FDD314A1268002AFD
:106204002EDB30490A60304A1268032A4ED8DFE890
:1062140002F00211151B4FF090424FF000419161C2
:1062240002F580624FF48011916127490A680132B6
:106234000A6010E0254A10219161F6E74FF0904280
:106244004FF400419161F0E7204A4FF480119161CD
:106254001D4A00211160013B184AC2F8A030704762
:10626400524218490A60184A1268032A1ED8DFE805
:1062740002F0020D13174FF090424FF0004191616C
:1062840002F580624FF480119161CEE74FF09042A5
:106294004FF400419161C8E70C4A10219161C4E7B1
:1062A4004FF090424FF000419161D1E706490A68EE
:1062B40001320A60032ACBDCCDE770474832002064
:1062C400646800208868002070680020000400488A
:1062D40070B50023194A1360194A1360194A1360F0
:1062E400194C1A4D1A4E08E0FFF7AAFD0CE0FFF70F
:1062F40093FE13E0FDF70CFBF8B9236F23B12B6871
:1063040013B13368002BEFD0D4F8883033B1114B7C
:106314001B681BB1104B1B68002BE8D0D4F8A030CD
:10632400002BE7D00D4B1B68002BE3D00C4B1B68F4
:10633400002BDFD1FFF75CFFDCE770BD4C68002069
:1063440050680020D8680020483200206C68002083
:1063540090680020686800208C6800206468002031
:046364008868002025
:10636800F8B52A4A136853F80409294908601360E4
:106378000D46284C284E294F0EE0FFF75FFD16E02A
:10638800FFF748FE1DE0FFF731FF254B1B68022B86
:1063980024D0244B1B682BBB2B6813B3FAF728F8BF
:1063A800236F23B1336813B13B68002BE5D0D4F8D1
:1063B800883033B11C4B1B681BB11C4B1B68002B6E
:1063C800DED0D4F8A030002BDFD0194B1B68002B8F
:1063D800DBD0184B1B68002BD7D1D4E7104B002219
:1063E8001A60F8BDFDF792FA012806D0022807D0F6
:1063F800114B1B68002BCFD0F3E7FDF7F9FDF7E74A
:106408000D4A136843F480731360EAE79468002028
:10641800B8680020483200206C680020906800208E
:106428005468002038020020686800208C6800202A
:0C6438006468002088680020D068002004
:1064440008B5054B1A681368642101FB03F3136054
:0C645400FFF788FF08BD00BF946800201F
:1064600008B5474B1B6863B1464B1B684BB1454BA6
:1064700000221A60444A1368191D1160434A1268C9
:106480005A60434BD3F8A030B3F1FF3F36D0414BB5
:106490001B68BBB9404A1360404A13604FF09043F9
:1064A0001A6822F040421A601A6842F080421A606C
:1064B00003F580631A6822F440721A601A6842F485
:1064C00080721A6030490B6853F804293148026021
:1064D0000B606AB94FF090434FF000429A6103F5A8
:1064E00080634FF480129A61294B0022C3F8A020E8
:1064F0002A4B00221A60FFF77DFE08BD254B0022C3
:106500001A604FF090431A6822F040421A601A68ED
:1065100042F080421A6003F580631A6822F44072E8
:106520001A601A6842F480721A60174B1A6813686E
:10653000002B0BDD4FF090434FF000429A6103F5C2
:10654000806310229A61FEF7EBFCD6E7002B0ADB92
:106550004FF090434FF000429A6103F580634FF48F
:1065600080129A61EFE75B4213604FF090434FF463
:1065700000429A6103F580634FF480129A61E2E76A
:10658000CC680020E868002094680020E4680020BF
:10659000483200206468002070680020886800206D
:1065A00038B58C280AD8174C04EBC00401E0FAF780
:1065B00051F814F8010B0028F9D122E0124B1B68A6
:1065C00003EB4301114A02EBC1021269904209D068
:1065D00003EB43020D4901EBC202013B183A11697A
:1065E0008142FAD103EB4303DB00084D5C1E2C44CF
:1065F0000F351D4414F8010F18B1FAF72BF8AC420F
:10660000F8D138BD3C790008B0680020483200203D
:106610002DE9F04383B0924B93E803000090ADF86E
:106620000410904B1D6815B103B0BDE8F0838E4B8C
:106630001B688E4A1360D3F8009029F400278C4B16
:106640001E6806EB46060D20FAF704F846B12C4604
:106650004FF020084046F9F7FDFF0134A642F9D17A
:10666000824B188801F065FE2020F9F7F3FF1FFA2E
:1066700089F001F05EFE2020F9F7ECFF8D2F1AD88B
:106680003846FFF78DFF7C2F52D07D2F55D07E2FBF
:1066900079D07F2F7FD0802F56D0832F00F083803A
:1066A000822F00F0868029F4002929F00209B9F12F
:1066B000840F49D055E02D20F9F7CCFF3E20F9F7A3
:1066C000C9FF2020F9F7C6FF3846FFF769FF664B80
:1066D0001B68D3F80480A8F110047A2F75D07B2FA3
:1066E00000F08180772F00F09780624C604E032D80
:1066F00000F0A5802368022B40F2A180F9F77CFE10
:10670000FEF724F80028F2D0FDF704F90546012829
:1067100000F08C80022800F08C800428E7D13368D8
:10672000002B00F08C80544A136002232360DEE7C4
:10673000524B1B681B683BB1C9E7504B1B681A687A
:1067400053F8043C9A42C2D0684601F0CCFD464B57
:106750001B685868043080B201F0EBFD2920F9F77E
:1067600079FF792FB3D12820F9F774FF444B1B68C8
:10677000102B24D03C4B1B685868FAF7BDFD29202C
:10678000F9F768FFAEE73D4B1B6853F8042C1B6814
:106790009A42D9D29BE7394B1B6853F8042C1B68EB
:1067A0009A42D1D993E7354B1B681B68002BCBD19C
:1067B0008DE7324B1B681B68002BC5D087E72A4B3F
:1067C0001B68586801F0F7FDD9E72820F9F742FF68
:1067D000207820B1F9F73EFF0134A045F8D12920F7
:1067E000F9F738FF81E72820F9F734FF661E08F132
:1067F000FF3816F8010F18B1F9F72CFF4645F8D10C
:106800004020F9F727FF184B1B68988801F0D3FD4B
:106810002920F9F71FFF68E72020F9F71BFF3C202C
:10682000F9F718FF2D20F9F715FF5EE7FDF7E4FBF8
:106830005DE70C4A136843F480731360F4E620208C
:10684000F9F708FF723F022F03D8684601F04BFDAD
:10685000EAE67B20F9F7FEFE2020F9F7FBFEE3E6EF
:10686000707F0008D0680020C0680020BC6800204D
:10687000B468002038020020EC68002094680020F2
:046880005C68002030
:1068840008B5FFF7C3FE064B1B6843B9054B1B68ED
:106894001A68054B53F822309847FDF739FE08BDB6
:0C68A400D0680020C06800200000002028
:1068B00008B51A4A136801331360194B19680A1D89
:1068C0001A60184A13684B601B6823F40023136096
:1068D0001B6823F400228C2A0BD8134A1268022A60
:1068E00004D0124A52F82330984708BDFFF7CAFF78
:1068F000FBE70D4B1B68032B06D00D4B1B68002BD1
:10690000F3D1FFF7D5FFF0E7FFF782FE084B1B68D6
:10691000002BEAD1FDF7FEFDEFE700BFB4680020D1
:106920009C680020C0680020380200200000002081
:04693000D06800200B
:10693400F0B587B001AC494D0FCD0FC42B6823705F
:10694400474B1B68474A484E06EB8206B3427ED249
:10695400464D434C464F46E0FFF7A8FF4CE0FDF799
:10696400F3FE50B923681B688C2B18D82A68032AB5
:1069740012D057F8233098473EE0FCF7C9FF0128AE
:1069840007D00228EED13B4A136843F480731360A6
:106994005DE0FDF72FFBE5E7FFF772FF2CE02B68C6
:1069A400032B02D0FFF782FF26E0FFF72FFEFDF74F
:1069B400AFFDF7E7FFF744FA28E02F4BD3F8A030F8
:1069C40033B12E4B1B681BB12D4B1B68002B2DD0F4
:1069D400284B1B68002B3AD12368002B29D00433A1
:1069E4002360B34233D22A68002AB8D11B688C2BA7
:1069F400B2D857F8233098471F4B1B6F33B1214B44
:106A04001B681BB1204B1B68002BD3D01A4BD3F847
:106A14008830002BD1D01D4B1B68002BCDD01C4BD4
:106A24001B68002BC9D1FFF7F7FAC6E7FFF7E0FBB5
:106A3400CEE70E4B1B68032B0BD00C4B01221A60C4
:106A44000023144A1360144A1360144A136007B0F5
:106A5400F0BD01A801F045FCEFE700BF6C8200081F
:106A6400C0680020084200204802002038020020AC
:106A740000000020D0680020483200206468002014
:106A8400886800206C6800209068002068680020F6
:106A94008C680020CC680020E8680020B4680020DE
:106AA400F8B52D4B1C68002C33D12C4B1B6803EB21
:106AB40043012B4A02EBC102526912F0406F0CD021
:106AC400284A1168081D106003EB4303244A02EBB3
:106AD400C3031B694B602046F8BD214A02EBC10386
:106AE4001B6923F40023204A1360204B01221A60FF
:106AF4001F4D2F681F4C266852232B6023601E4BAA
:106B040000221A60FFF714FF2F6026601B4B1C68DD
:106B1400E1E7124B1B6803EB4301114A02EBC1028C
:106B2400546914F0406406D10D4A02EBC10318699C
:106B3400FDF712FACFE77A20FDF70EFA074B186833
:106B440000EB4000064B03EBC0001030FDF704FAE5
:106B54000A4B1C68BFE700BFD4680020A06800206F
:106B64004832002094680020C0680020CC680020CF
:106B7400506800204C680020D8680020D0680020AD
:106B840070B50023274A1360274A13601546274E21
:106B940009E07920FDF7E0F9254B1868FDF7DCF9E9
:106BA4002A68204B1A60234C2A6823689A4219D217
:106BB400FCF79EFF3378002BF6D0FDF745F858B16B
:106BC4001D4B1B68002BE4D11C4A1368191D11606E
:106BD400174A12685A60E3E7FDF7EAF838B1FFF79D
:106BE4005FFF00B170BD2A680E4B1A60DBE7FDF74A
:106BF400A1F848B1FDF7C8F9114B1B68002BF1D17E
:106C04002A68084B1A60CEE70D4A136843F0010363
:106C140013600C4B1A680C4B1A60034B1A68014B37
:106C24001A60DFE7446800204C680020F467002005
:106C34004868002050680020D46800209468002030
:0C6C4400D0680020DC680020E068002020
:106C50002DE9F04F93B00CACAA4D0FCD0FC495E8C1
:106C6000030044F8040B217007ACA74D0FCD0FC4EF
:106C70002B6824F8023B1B0C2370A44B03AC0FCBF6
:106C800007C42380A24B1A68A24B1A60FCF732FF9C
:106C9000FDF790F860B9FDF74FF828B99E4A1368E0
:106CA00043F001031360FCE00CA801F01CFBF8E0CA
:106CB000974B1A68974B1A6007A801F014FB974D81
:106CC000286800EB4000964C04EBC00001F073FB19
:106CD0000D20F9F7BFFC2B6803EB430204EBC20461
:106CE000246914F4002F17D024F400248D48241AAA
:106CF000A40803EB43038A4A02EBC3035B6913F066
:106D0000406840F0D180874B53F82430772B00F057
:106D1000B9800126834D2AE003EB4302804901EB51
:106D2000C2025469C4F30B04E3E70D20F9F792FCA7
:106D300046461CE001342820F9F78CFC55F8240065
:106D4000043080B201F037FB2920F9F783FC0136CB
:106D50002020F9F77FFC2020F9F77CFC013455F85E
:106D60002430772B00F08E800136072EDDD805EB1E
:106D7000840080B201F0DDFA3A20F9F76BFC55F897
:106D80002400FFF70DFC55F8243023F40023A3F171
:106D90007C020A2ACED9792B13D07A2B27D07B2BD1
:106DA00032D0782BD4D12220F9F754FC631C55F84B
:106DB00023900234B9F1000F5ED0CDF8048047462D
:106DC00048E001342820F9F745FC574B1B68102B8D
:106DD00008D055F82400FAF78FFA2920F9F73AFC81
:106DE0000136B5E755F8240001F0E5FAF5E701347E
:106DF0002820F9F72FFC55F8240001F004FB292086
:106E0000F9F728FC0136A3E701342820F9F722FC22
:106E100055F8240001F0F7FA4020F9F71BFC35F88B
:106E2000240001F0C8FA2920F9F714FC01368FE795
:106E30005C20F9F70FFC4FEA1B1001F052F80AF042
:106E40000F0001F04EF80837182F88BF4746B9F1F8
:106E5000010911D01FB955F8243001930134019B69
:106E600023FA07FA5FFA8AFBABF120035E2BDFD827
:106E70005846F9F7EFFBE6E7013C2220F9F7EAFB79
:106E8000033665E7274800EB840080B201F051FA31
:106E90003A20F9F7DFFB3B20F9F7DCFB0D20F9F78F
:106EA000D9FB13B0BDE8F08F03A801F01CFA1E4B0C
:106EB0001B68102B1BD0194B1B6803EB4303184AAC
:106EC00002EBC303186901F056F82020F9F7C2FB62
:106ED0004020F9F7BFFB114B1B6803EB430310483D
:106EE00000EBC300103080B201F065FAD6E70B4B1F
:106EF0001B6803EB43030A4A02EBC303186901F062
:106F00005AFAE2E7847F00089C7F0008B07F0008FF
:106F10004C68002044680020D0680020A068002051
:0C6F200048320020480200205C6800207D
:106F2C0038B51B4C1B4D2B682360FCF7DDFD2B6823
:106F3C002360194B1B6823B35D1E03EB4303174CF3
:106F4C0004EBC304193C06E0284638BD013D183C4F
:106F5C00B5F1FF3F18D0124901F1100EA4461CF8F0
:106F6C00010F11F8013BA3F16102D2B2192A9CBFA7
:106F7C00203BDBB28342E9D10028E5D07145EED14C
:106F8C00E4E74FF0FF30E0E74FF0FF30DDE700BF04
:106F9C00446800204C680020B06800204832002073
:046FAC00F467002066
:106FB00038B5FFF7BBFFB0F1FF3F0FD0044600EB41
:106FC0004003294A02EBC3035B6913F0406F0BD007
:106FD000264A136843F08003136038BD234A1368C0
:106FE00043F021031360F8E7FFF7A0FFB0F1FF3F84
:106FF00027D000EB40031C4A02EBC3035B6913F08C
:10700000406F24D1844228D3174B04EB440403EB94
:10701000C404256945F4002500EB400203EBC202DD
:1070200014691561124B134A1268191D01EB820194
:1070300053F8042BA24208BF43F8045C8B42F7D1FB
:10704000CBE70A4A136843F021031360C5E7074AF8
:10705000136843F080031360BFE7044A136843F0EA
:1070600080031360B9E700BF48320020D0680020D9
:0870700048020020DC6800204A
:1070780010B5FFF757FFB0F1FF3F24D000EB4003F6
:10708800174A02EBC30319695B69C3F30B03154C79
:1070980004EB830421F40023A3421AD900EB400037
:1070A8000F4B03EBC00004610E4B0F4A1268181D0A
:1070B80000EB820053F8042B8A4208BF43F8044CC3
:1070C8008342F7D110BD094A136843F021031360C6
:1070D800F8E7064A136843F080031360F2E700BF3D
:1070E8004832002048020020DC680020D0680020D8
:1070F80010B58AB00DF10C0C114C0FCCACE80F0098
:1071080094E80700ACE803002CF8022B120C8CF86A
:1071180000200C4A6B4607CA03C31A8003A801F073
:10712800DEF8FAF7F1F90028FBD0C3B2592B02D1E7
:1071380001200AB010BD684601F0D1F80020F8E738
:08714800D07F0008EC7F000875
:1071500070B592B005460DF1040C3B4C0FCCACE879
:107160000F000FCCACE80F000FCCACE80F00236889
:107170002CF8023B1B0C8CF80030344C344E336836
:107180002360FCF7B7FC33682360FCF75FFD38B180
:10719000304A136843F080031360002012B070BDC2
:1071A0000446FCF7C9FD30B92B490DF1380C01F14B
:1071B000100E60460FE001A801F095F8FFF79CFF64
:1071C00000283FD00D20F9F745FAEDE710F8013C13
:1071D00073B171450CD011F8013B00F8013BA3F1EC
:1071E0006102D2B2192AF1D8203B00F8013CF0E745
:1071F00000238DF847309DF838307BB1174A11686D
:1072000001EB4101164A02EBC102013A02F8013FCB
:1072100001341CF8013F0BB10F2CF7D10F4B1B6849
:107220000F4A03EB430002EBC000044400216170ED
:107230000C4909680C4C04EB810404612943416149
:107240000120ABE70220A9E7808200084468002003
:107250004C680020D0680020F4670020B06800204F
:0C72600048320020E068002048020020B6
:10726C0038B54FF04060FFF76DFF78B10A4C0B4812
:10727C000368226852F8045903EB430C084901EBEC
:10728C00CC010D6122600133036038BD054A1368DF
:10729C0043F001031360F8E794680020B068002005
:0872AC0048320020D0680020E8
:1072B40008B50020FFF74AFF40B1022807D0084B69
:1072C4001A68084B1A60084B01221A6008BD074B64
:1072D4001B6803EB4303DB00054A0021D154F5E7A7
:1072E400E0680020DC680020D4680020B06800203A
:0472F40048320020FC
:1072F80030B583B01F4B93E8030000908DF804105D
:107308001D4A136853F804491360052C06D91B4A13
:10731800136843F48063136003B030BD684600F01F
:10732800DEFF174800F0DBFF04F13000C0B2F9F7C8
:107338008DF9D4B12020F9F789F93F20F9F786F9BA
:10734800FFF7D6FE0028E7D00E4D2C60F9F7A6F817
:107358002B68002BE0D0F9F763FB0028DCD1074A43
:10736800136843F020031360D6E7074800F0B7FF1F
:10737800E0E700BFB482000894680020D0680020CD
:0C738800D88200080C690020C4820008B4
:1073940030B583B0224B93E8030000908DF80410BD
:1073A400204A136853F804491360052C06D91E4A71
:1073B400136843F48063136003B030BD684600F083
:1073C40090FF1A4800F08DFF04F13000C0B2F9F7C5
:1073D4003FF974B12020F9F73BF93F20F9F738F968
:1073E400FFF788FE0028E7D0114B1C60F9F75EF91F
:1073F400E2E7104800F075FF2020F9F729F93F2053
:10740400F9F726F9FFF776FE0028D5D0084C0025B9
:107414002560FDF7EDF8F9F719F82560CCE700BF12
:10742400BC82000894680020D0680020D88200083C
:087434000C690020C48200086D
:10743C004FF0FF0C1CEAD0521EBF1CEAD153FF2A9E
:10744C00FF2B28D01A444FF0004C90EA010313EAAA
:10745C000C034CEA01214CEA0020A0FB01C1B1F164
:10746C00004F62F17F0238BF49004CEA416CFE2AA2
:10747C0009D253EA11204CEAC07C28BFBCF10103AD
:10748C0040EBC2507047124244BF18467047FF2071
:10749C0043EAC050704710EACC5F08BF00F00040D0
:1074AC0011EACC5F08BF01F000410CEAD153FF2A6E
:1074BC0018BFFF2B03D0484000F000407047002855
:1074CC001EBFB0F1004F0029B1F1004F11D0FF2ABF
:1074DC0002D15FEA402C0CD1FF2B02D15FEA412C88
:1074EC0007D1484000F0004040F0FE4040F400005E
:0C74FC0070474FF0FE4040F44000704725
:10750800FF2313EAD0521EBF13EAD153FF2AFF2BE1
:1075180036D0D21A7F3281EA000C0CF0004C4FF0C2
:10752800004343EA002043EA012130B4431A3CBF38
:1075380001EB4303013A090AB3FBF1F505FB1133EB
:107548001B02B3FBF1F001FB103300EB05201B021B
:10755800B3FBF1F505EB00205CEA500050EBC2509C
:1075680030BC002A09DDFF2A38BF70474FF07F4042
:107578000CF0004C4CEA500070470CF0004070478B
:1075880003EAD15393F0FF0F08D192F0FF0F1BD0FD
:107598005FEA412C14D04FF440001DE092F0FF0F39
:1075A80005D14FF07F43B3EB400F10D00CD193F0CF
:1075B800000F08BF92F0000F06D093F0000F06D01E
:1075C800484000F0004070474FF4400004E0484055
:1075D80000F0004040F4000040F0FE40704700BF5B
:1075E8004FF4001C1CEB410F98BF1CEB430F11D844
:1075F80051EA030C50EA4C0C5CEA020C0AD004D2A3
:1076080082428B418041404270479042994180417B
:0876180040427047002070475A
:107620004FF4001C1CEB410F98BF1CEB430F11D80B
:1076300051EA030C50EA4C0C5CEA020C0AD004D26A
:107640009042994180414042704782428B41804143
:08765000404270470020704722
:10765800C0F3C751D1F19E0108D950F400004FEA98
:10766800002020FA01F048BF404270474200B2F1C2
:107678007F4F88BF20F0004010F0004058BF6FF0E7
:047688000040704707
:10768C0010F0004118BF4042B0FA80F210FA02F339
:10769C000DD0D2F19D0241EAC25101EB13205A06E2
:1076AC0038BF704700F1010008BF20F0010070479F
:1076BC00C0F3C75191B142004FEA40704FEAD2017A
:1076CC004FEA310101F16051B2F17F4F38BF704781
:1076DC0001F1605118BF41F40021704710F00041D6
:0476EC0000207047C3
:1076F0000000000000000000010203040607080962
:087700004B65726E656C3A00E6
:107708000000000000000000000000000000000071
:107718000000000000000000000000000000000061
:107728000000000000000000000000000000000051
:107738000000000000000000000000000000000041
:107748000000000000000000000000000000000031
:107758000000000000000000000000000000000021
:107768000000000000000000000000000000000011
:107778000000000000000000000000000000000001
:1077880000000000000000000000000000000000F1
:1077980000000000000000000000010000000500DB
:1077A80000000000000000000000000000000000D1
:1077B80000000000000000000000000000000000C1
:1077C80000000000000001000000040000000400A8
:1077D80000000000000000000000000000000000A1
:1077E8000000000000000400000004000000040085
:1077F8000000040000000400000000000000000079
:107808000000000000000000000000000000000070
:107818000000000000000000000000000000000060
:107828000000000000000000000000000000000050
:10783800000000000000000000000000000004003C
:107848000000040000000400000000000000000028
:10785800000000000000000000000000000004001C
:107868000000000000000500000005000000050001
:1078780000000400000004000000040000000400F0
:1078880000000000000001000000010000000100ED
:1078980000000100000003000000030000000300D6
:1078A80000000300000003000000030000000300C4
:1078B80000000300000003000000030000000300B4
:1078C80000000300000002000000020000000200A7
:1078D800000002000000020000000100000001009A
:1078E8000000080000000800000008000000080070
:1078F8000000080000000800000008000000080060
:10790800000008000000080000000800000008004F
:107918000000080000000800000008000000020045
:107928000000020000000100000005000000010046
:04793800000001004A
:10793C004552524F5200000044524F50000000007C
:10794C004455500000000000535741500000000007
:10795C004F56455200000000524F540000000000EA
:10796C002D524F54000000005049434B00000000C2
:10797C00524F4C4C00000000494E4A454354000005
:10798C002B00000000000000312B00000000000064
:10799C002D00000000000000312D00000000000050
:1079AC004142530000000000534849465400000077
:1079BC00414E4400000000004F5200000000000047
:1079CC00584F5200000000004E4F540000000000C1
:1079DC002B2F2D00000000002A00000000000000EA
:1079EC002F000000000000002A2F00000000000003
:1079FC004D4F4400000000002F4D4F44000000008C
:107A0C00425345540000000042434C520000000019
:107A1C00425453540000000052414E444F4D00005C
:107A2C003D3D000000000000213D00000000000072
:107A3C003E000000000000003E3D00000000000081
:107A4C003C00000000000000553C0000000000005D
:107A5C003C3D000000000000303D00000000000034
:107A6C00564152434F4E0000524556000000000054
:107A7C005700000000000000520000000000000051
:107A8C0041525241590000004B45593F0000000043
:107A9C004B45590000000000454D495400000000C2
:107AAC002E000000000000002E4800000000000026
:107ABC002E440000000000002E22000000000000F8
:107ACC00445A00000000000048580000000000006C
:107ADC00584E4F50000000004D53000000000000B5
:107AEC0044530000000000005449580000000000FE
:107AFC0054494D45000000004652455131320000BA
:107B0C0050574D310000000050574D32000000001E
:107B1C00465245513300000050574D3300000000D1
:107B2C004F480000000000004F4C00000000000017
:107B3C0044414F340000000044414F350000000028
:107B4C00495055000000000049504400000000005E
:107B5C00495A0000000000005244494E0000000049
:107B6C005241444300000000494E492D53504900F6
:107B7C005350490000000000494E492D4932430042
:107B8C0049545831000000004954584E0000000080
:107B9C0049525831000000004952584E0000000074
:107BAC0049525841444E00004D4F543100000000E2
:107BBC004D4F5432000000004D4F54330000000074
:107BCC005245475700000000524547520000000044
:107BDC00524547425345540052454742434C52008C
:107BEC0052454742545354002E53000000000000ED
:107BFC0046530000000000004F50530000000000EE
:107C0C00555345520000000053454500000000004C
:107C1C004D454D00000000005354000000000000D2
:107C2C0052554E00000000004E4F2D4442470000BC
:107C3C004445425547000000464F5247455400000A
:107C4C0041424F52540000005245504C41434500B4
:107C5C00524553544F524500494600000000000065
:107C6C0043415345000000003C4341534500000094
:107C7C003E43415345000000454C53450000000075
:107C8C005448454E00000000444F00000000000026
:107C9C00554E54494C0000005748494C45000000D3
:107CAC00414741494E000000464F52000000000081
:107CBC004C4F4F5000000000490000000000000035
:107CCC00434F4E5449000000425245414B000000C6
:107CDC005A425245414B000052455455524E0000F9
:107CEC003A000000000000003B0000000000000013
:107CFC00646F535452000000646F4C4954000000F0
:107D0C00646F56414C554500646F52455600000057
:107D1C00646F494600000000646F43415345000006
:107D2C00646F3C4341534500646F3E4341534500EF
:107D3C00646F454C53450000646F444F00000000D5
:107D4C00646F554E54494C00646F5748494C45007C
:107D5C00646F414741494E00646F464F520000002A
:107D6C00646F4C4F4F50000052502D3100000000FA
:107D7C0052502D34000000004155544F45584500D9
:107D8C003F00000000000000534156450000000079
:087D9C004C4F414400000000BF
:107DA400FEE7FEE7FEE7FEE7FEE7FEE7FEE7FEE7A7
:107DB400FEE7FEE7FEE7FEE7FEE7FEE7FEE7FEE797
:107DC400FEE7FEE7FEE7FEE7FEE7FEE7FEE7FEE787
:107DD400FEE7FEE7FEE7FEE7FEE7FEE7FEE7FEE777
:107DE400FEE7FEE7FEE7FEE7FEE7FEE7FEE7FEE767
:107DF400FEE7FEE7FEE7FEE7FEE7FEE7FEE7FEE757
:107E0400FEE7FEE7FEE7FEE7FEE7FEE7FEE7FEE746
:107E1400FEE7FEE7FEE7FEE7FEE7FEE7FEE7FEE736
:107E2400FEE7FEE7FEE7FEE7FEE7FEE7FEE7FEE726
:107E3400FEE7FEE7FEE7FEE7FEE7FEE7FEE70348B0
:107E44008546F9F72FFC00F003B870470080002046
:107E540011488546114C20680434004201D0804703
:107E6400F9E70F480F49091A082903DB00220260C9
:107E7400043001600C480D49884205D00268043082
:107E840003B4904703BCF7E700208646EC46002085
:107E94000021074A9047FEE7008000202084000864
:107EA40020690020206D00204580000845800008DE
:047EB400CD080008ED
:107EB8001EF0040F0CBFEFF30880EFF309800149AF
:087EC800084700004780000894
:107ED000756E646572666C6F77212000202D2D2DE4
:027EE000200080
:107EE20008B5024600F13003D8B2392884BF02F146
:0A7EF2003700C0B2F8F7ADFB08BD81
:107EFC00313238205352414D2062797465732833E6
:107F0C003220776F72647329207374617274696E96
:0A7F1C00672066726F6D2030780058
:107F260010B50446000FFFF7D9FFC4F30360FFF74F
:107F3600D5FFC4F30350FFF7D1FFC4F30340FFF7A7
:107F4600CDFFC4F30330FFF7C9FFC4F30320FFF7E7
:107F5600C5FFC4F30310FFF7C1FF04F00F00FFF7DE
:0A7F6600BDFF2020F8F773FB10BDEB
:067F70002849502D3E00DF
:0E7F760008B5F9F7BEF92020F8F769FB08BD41
:107F840063616E277420534545204B65726E656CA2
:107F9400204F70730000000055736572486561647A
:107FA40065725F5374727563743D00005661724369
:0A7FB4006F6E3A56616C75653D0072
:107FBE0010B504462020F8F746FB2046F9F795F950
:027FCE0010BDE4
:107FD00020636F6E6669726D20772E7570706572A2
:107FE00020636173652027592720000063616E6359
:067FF000656C6C65640085
:027FF600FEE7A4
:107FF800203C2D6E6F742061204B65726E656C207D
:108008004F50206E6F722061206E756D6265720030
:10801800203C2D696E76616C696420666F7220421F
:1080280061636B2D4374726C00000000203C2D527C
:0D803800756E74696D65204572726F72007F
:108046004FF0E023D3F82C3D002B00DBFEE74FF08A
:10805600E022D2F82C3D43F00043C2F82C3D836960
:0680660002338361704744
:10806C0043466F72746820666F722053544D3332DE
:10807C0047343331204E75636C656F2076000000F9
:10808C002020286329323032302D323420572E53A1
:10809C006368656D6D657274000000002020537973
:0B80AC007374656D436C6F636B3D00E7
:1080B800537461636B3D0000436F64655468726577
:1080C80061643D00456D70747920000050726F6ADC
:1080D80065637400206C6F616465642020204155DD
:1080E800544F4558453D00004672657131323D0098
:1080F800487A2050574D313D000000002C50574D14
:10810800323D0000202046726571333D00000000BA
:10811800487A2050574D333D000000004D4F5431F0
:108128003A0000002020204D4F54323A0000000051
:108138002020204D4F54333A0000000053746570DE
:108148003D0000006D73204E5354503D0000000068
:0781580044432F50574D0076
:108160004572726F722300002028636F6C2000003C
:10817000206E6F7420666F756E6400005F53796EB9
:1081800074617820457272005F537461636B20459F
:10819000727200005F436F6D70696C65206F6E6C6A
:1081A000790000005F4E6F20492F4F20436F6D6DA7
:1081B00020416363657373005F496E76616C696427
:1081C00020436F6465206163636573730000000082
:1081D0005F6F7574206F6620436F6E7465787400EE
:1081E0005F52756E74696D65206F6E6C7920746F67
:1081F0006B656E005F5468726561642063616E63D5
:10820000656C6C65640000005F4E756D6265722080
:108210006F7574206F662052616E67650000000004
:108220005F4469766973696F6E206279205A65725E
:108230006F0000002020636F6D70696C696E672E9F
:038240002E2E00DF
:1082440020202841444320696E697469616C697A0D
:108254006564292000000000202028414443206F49
:05826400666629200000
:10826C002064656275672066696E69736865642051
:01827C000001
:10828000205761726E696E673A2077696C6C206F57
:1082900076657272696465204B65726E656C204FFD
:1082A0007020776974682073616D65206E616D65FB
:0382B0002120008A
:0582B400536176650036
:0582BC004C6F6164003D
:1082C400283D456D7074792050726F6A6563742916
:0182D40000A9
:0D82D8002050726F6A656374206E6F2E0077
:1082E60010B5044614F8010B28B1F8F7B0F914F8E4
:0882F600010B0028F9D110BDB5
:1082FE0010B50446C0F3031303F13000392888BFCC
:10830E0003F13700F8F79FF904F00F0404F1300081
:10831E00392888BF04F13700F8F795F92020F8F7CF
:04832E0092F910BDF3
:1083320010B50446000F1ED1C4F3036014F0706F31
:108342001DD1C4F3035014F4700F1CD1C4F30340C5
:1083520014F4702F1BD1C4F3033014F4704F1AD1EC
:10836200C4F3032014F4706F19D1C4F3031014F092
:10837200F00F1AD017E0FFF7B3FDC4F30360FFF765
:10838200AFFDC4F30350FFF7ABFDC4F30340FFF7A7
:10839200A7FDC4F30330FFF7A3FDC4F30320FFF7E7
:1083A2009FFDC4F30310FFF79BFD04F00F00FFF7DE
:0483B20097FD10BD66
:1083B60010B504463020F8F74AF97820F8F747F95F
:0883C6002046FFF7B3FF10BDD4
:1083CE002F2810D9A0F13003DBB2092B09D90A29C5
:1083DE000CD0A0F14103DBB2052B0AD83738C0B25E
:1083EE007047184670474FF0FF3070474FF0FF3020
:0883FE0070474FF0FF3070479B
:1084060038B50546A0F11004207820B1F8F71FF919
:088416000134A542F8D138BD84
:108420008986000848020020D16600009F86000867
:108430000000002040840008480200000000000006
:1084400045170008551700087D170008A9170008F0
:10845000C1170008D5170008F91700081D180008F3
:1084600061180008C9180008311900084D190008E2
:108470005D19000879190008891900089D1900087C
:10848000E5190008011A00081D1A0008391A000829
:10849000491A0008D9010008591A000859020008B1
:1084A0008D1A0008C51A0008F91A0008311B0008C7
:1084B0006D1B0008B11B0008C91B0008ED1B00085C
:1084C000211C0008451C0008691C00088D1C0008C0
:1084D000B11C00080D1C00086D7200083541000831
:1084E000D51C0008111D0008451D00087147000833
:1084F000892B0008E12A0008012C0008E12B000864
:10850000252E0008E9470008951D0008B51D000844
:10851000D51D00086963000845640008F91D0008BE
:10852000191E0008B54C0008AD4B0008094D0008A5
:10853000D14E0008214F00089D500008D551000879
:108540003D2E0008A52E00080953000825540008F8
:1085500041550008B14F00089D570008F95A00081E
:108560003D5B0008491E0008291F0008E11F0008A4
:10857000D52000088D21000871220008195F00082D
:10858000F160000861640008E12300081924000874
:10859000492400089D240008F1240008492C000803
:1085A000792600080D2F0008152D0008516C0008D1
:1085B000BD2F000899260008A5260008B12600084E
:1085C000F92A0008393E0008BD260008B16F0008EE
:1085D00079700008054200082D4200085542000845
:1085E0007D420008A54200084D250008E142000830
:1085F000094300085143000899430008E14300087B
:10860000094400087D25000899250008C9250008AF
:10861000DD25000805260008B57200085144000851
:10862000392B00081D2800083D2800085D28000897
:1086300081280008AD280008D9280008052900086D
:10864000312900084129000861290008A5290008EE
:10865000E9290008052A0008412A0008C12A000863
:10866000D12A0008093F0008AD300008F97200085F
:10867000957300080A00000001000000A8510020C6
:088680004C6500200024F40009
:10868800206861680834094204D000220270013071
:068698000139FBD170471F
:10869E0020686168A2680C34124205D00B78037012
:0A86AE0001300131013AF9D17047A3
:0400000508007E432E
:00000001FF
